:100000000C9466000C9487000C9487000C94870075
:100010000C9487000C9487000C9487000C94870044
:100020000C9487000C9487000C9487000C94870034
:100030000C9487000C9487000C9487000C94870024
:100040000C9487000C9487000C9487000C94870014
:100050000C9487000C9439030C9487000C9487004F
:100060000C9487000C94D8120C9487000C94870091
:100070000C9487000C9487000C9487000C948700E4
:100080000C9487000C9487000C9487000C948700D4
:100090000C94BC1A0C9487000C9487000C94870075
:1000A0000C9487000C9487000C9487000C948700B4
:1000B0000C9487000C9487000C9487000C948700A4
:1000C0000C9487000C9487000C94870011241FBEA9
:1000D000CFEFD1E2DEBFCDBF00E00CBF14E0A0E067
:1000E000B2E0E0ECF3E900E00BBF02C007900D9234
:1000F000AC33B107D9F717E0ACE3B4E001C01D920F
:10010000A133B107E1F70E94890C0C94DE490C94ED
:100110000000109242048091420480934104809137
:100120004104809340048091400480933F041092E6
:10013000430410925004109251040895EEE6F0E04A
:1001400080818260808383E084BD85BD8AEF87BD26
:1001500008950895089580917100817008959B011C
:10016000AC01CA01AA27BB27BC01892B79F0687FA3
:10017000672B59F483E056954795379527958A95CF
:10018000D1F73093A5042093A40408953093A504D7
:100190002093A40408958091A204982F9295969597
:1001A00096959370282F221F2227221F9227282FEF
:1001B00022952F709227282F2695269592279170A9
:1001C000880F892B8093A2040895909394048093C0
:1001D000930485EB9BE39093AC048093AB0483E39F
:1001E00093E19093B2048093B10485E694ED9093EB
:1001F000A7048093A6040895809193049091940499
:10020000AC01440F452F441F550B519548275927E2
:100210006091AB047091AC04709394046093930468
:100220008091B1049091B2049093AC048093AB049C
:100230002091A6043091A7043093B2042093B10416
:10024000C9010024969587950794969587950794FC
:10025000982F802D8227932784279527542F442772
:100260005295550F507E842795279093A70480932D
:10027000A604660F771F6F5F7F4F869F9001879F51
:10028000300D969F300D1124C9010895FC01908115
:10029000992351F08091C80085FFFCCF9093CE0048
:1002A000319690819923B1F708951F93CF93DF93EF
:1002B000182F492FE0E1F7E2C0E0D0E0812F942F22
:1002C000BF010E9495499B016115710589F5812F38
:1002D000942FBF010E949549182F492FCF016AE042
:1002E00070E00E949549FB012196C430D10531F799
:1002F0003097A1F18091C80085FFFCCF812F942F0A
:10030000BF010E949549605D6093CE00CF016AE015
:1003100070E00E9495499B0161157105F9F0812FEC
:10032000942FBF010E949549182F492FF901E2CF60
:100330008091C80085FFFCCF822F805D8093CE0026
:10034000812F942FBF010E949549182F492FCF016B
:100350006AE070E00E949549FB01CACFDF91CF911E
:100360001F910895982F9F709A3040F48091C80093
:1003700085FFFCCF905D9093CE0008958091C800DA
:1003800085FFFCCF995C9093CE000895CF93DF93C7
:10039000EC01892F992782958F700097C1F48D2FDA
:1003A0009927009789F4CE01929582958F708927BD
:1003B0009F708927009711F00E94B2018C2F0E9434
:1003C000B201DF91CF9108950E94B201ECCF0E945B
:1003D000B201E5CF982F8091C80085FFFCCF9093A4
:1003E000CE0080E090E008952091C800332727FDDB
:1003F00030952227330F221F3327C901089580919A
:10040000C80087FFFCCF8091CE0090E008959C014A
:100410008FEF8093980493E0283E390768F5809326
:1004200095048093960424363105D8F0C90164E61A
:1004300070E00E94954960939504C9016AE070E0FC
:100440000E949549CB016AE070E00E949549809333
:100450009604C9016AE070E00E9495498093970470
:1004600008952A30310548F7C9016AE070E00E941A
:1004700095498093970408951092950410929604DC
:1004800010929704089590914404936090934404CB
:1004900080934504089580914404836080934404CC
:1004A0000895F999FECF92BD81BDF89A30B5F999BA
:1004B000FECF019692BD81BDF89A20B5932F80E0C2
:1004C00030E0282B392BC9010895F999FECF92BD50
:1004D00081BDF89A80B50895F999FECF92BD81BD8E
:1004E00060BDF894FA9AF99A78940895FF920F9360
:1004F0001F938C01F62E672F0E946C02C801019693
:100500006F2D0E946C021F910F91FF9008958091B2
:10051000C90088618093C90083E38093CC00109266
:10052000CD008091C80087FD34C08091C9008068EB
:100530008093C9008091C10088698093C1008FE1D8
:100540008093C4001092C50090EC91B98CE382B9FD
:1005500087E384B995B99FEF97B988EF8AB98BE0A3
:100560008BB982E08DB99EB910BA91BB88E183BB8B
:1005700087EE84BB8DB581608DBD81E58CBD08950E
:100580008091CE008AE00E943C0F8091C80087FFD6
:10059000CCCF8091C80087FDF3CF8091C80087FF42
:1005A000F8CFEECFEF92FF920F931F93CF93DF938D
:1005B000EC0181E0CD32D80708F440C0CCE2D1E0B4
:1005C0007E0100E010E080918F04909190048C17E0
:1005D0009D0719F0CE010E94771AD0939004C09322
:1005E0008F04D093A104C093A0046091090270917C
:1005F0000A0280910B0290910C02A80197010E94BF
:10060000BC496FEF7FEF8FEF9FEF0E94BC49CA019B
:10061000B90128EE33E040E050E00E946A4960935F
:100620009C0470939D0480939E0490939F04DF919B
:10063000CF911F910F91FF90EF900895C431D10594
:1006400008F0BECFC4E1D0E054E1E52EF12C012D3D
:10065000112DB9CF85E090E00E9451020E94D20294
:1006600080918F04909190049093A9048093A804A2
:1006700008951F920F920FB60F920BB60F9211248E
:100680002F933F934F935F936F937F938F939F939A
:10069000AF93BF93EF93FF9340B1427090B18091BD
:1006A000AF04481749F1892F8170442309F4D8C059
:1006B000882309F4D8C09FEF8091F8038823D1F0F4
:1006C00080914B04882309F405C1913009F022C1BF
:1006D0008091A0049091A10407969093A104809327
:1006E000A0048D52914030F08CE291E09093A104EF
:1006F0008093A0044093AF0480915F048F3F29F062
:1007000080915F048F5F80935F04809160048F3FCE
:1007100029F0809160048F5F8093600480918A0447
:1007200090918B048F5F9F4F49F080918A04909144
:100730008B04019690938B0480938A0480916E04BD
:1007400090916F048F5F9F4F49F080916E0490915C
:100750006F04019690936F0480936E0480914E0411
:10076000882351F080914E04815080934E048091F3
:100770004E04882309F48AC080913C04823009F435
:100780008BC0813009F471C0882309F056C0809174
:10079000010290910202A0910302B09104028093A1
:1007A000050290930602A0930702B09308022091DD
:1007B00001023091020240910302509104028091A3
:1007C0009C0490919D04A0919E04B0919F04820F7F
:1007D000931FA41FB51F8093010290930202A09360
:1007E0000302B09304022091010230910202409171
:1007F0000302509104028091050290910602A0919B
:100800000702B0910802281739074A075B07A8F4C6
:1008100080914D048F5F80934D0480914D048170D1
:1008200080934D0480914C048F5F80934C048091A1
:10083000A0049091A1040E94D202FF91EF91BF9178
:10084000AF919F918F917F916F915F914F913F9168
:100850002F910F900BBE0F900FBE0F901F90189509
:10086000882309F428CF91E027CF99B19295917010
:1008700080915D04981709F390934D0490935D0463
:1008800080914C048F5F80934C04D7CFA4988091C3
:100890003C04823009F075CF8091590490915A043C
:1008A000892B59F28091590490915A0401979093A1
:1008B0005A04809359048091590490915A04892BC9
:1008C00009F0BBCF10924D0480914C048F5F809350
:1008D0004C04B3CF292F332727FD30958091A004F6
:1008E0009091A104280F391F3093A1042093A004F4
:1008F00081E02D32380708F0F7CE2431310508F0B9
:10090000F9CE84E190E09093A1048093A0044093F9
:10091000AF04F2CE9F3F09F0EDCE8091A0049091FC
:10092000A10407979093A1048093A004449708F032
:10093000E1CEE7CFCF92DF92EF92FF920F931F931A
:10094000CF93DF93F89480913C04813009F4C8C4BC
:1009500080918604813009F4A4C280913F048C30D8
:1009600060F010923F04809140048F5F80934004B8
:10097000809141048F5F80934104809141048823DA
:1009800041F08091410490E083709070892B09F4CC
:100990003EC280914204883038F010924204809127
:1009A0003C04882309F412C2809141048F70809323
:1009B000410490914004809100029817C0F0109279
:1009C0004004809143048F5F8093430490914304DB
:1009D0008091B004981708F044C28091440482606A
:1009E00080934404809148048160809348048091FE
:1009F0002B07882329F480914004882309F427C217
:100A000080914004882329F480918604823009F47F
:100A100097C2909150048091AA04981710F01092F8
:100A2000500480912B07882329F08091500488235B
:100A300009F4F3C18091EE048C3009F4F7C1809180
:100A40003C04882309F0F3C0909158048091F50389
:100A5000981710F0109258048091580480FFE1C05C
:100A60005C98809187042091F5034091F50390E014
:100A700030E0240F311D8217930714F01092870481
:100A8000809187046091F50366950E9489499923B6
:100A900009F4DDC0DD248091F50390915104869521
:100AA000899F202D1124921710F0109251048091EB
:100AB0002B07882349F080915104882309F4A39AD5
:100AC0002695821709F44AC28091EE04873009F412
:100AD000CEC0883008F4C3C08B3009F4C8C08C3055
:100AE00008F43EC28C3009F46EC38D3009F4BFC0E7
:100AF00080918604823009F4E4C380912B07882317
:100B000021F082E0D81609F4E7C380912B078823EF
:100B100009F408C2809173048F70809373048091EC
:100B2000410490E08370907002970CF4F7C185E265
:100B30000E9490168091730490E0837090700297E9
:100B40000CF4E9C18FEF80936B0480917C048823BF
:100B500009F0B1C180918504882371F0809145042A
:100B6000882351F08091AD04813009F4E6C2809170
:100B7000AD04882309F417C280914604882309F044
:100B800073C180914B04882349F080913C048823F1
:100B900029F48091F803882309F0DFC20E946718C6
:100BA000DD2031F080913D048F5F817080933D04A2
:100BB000809187048F5F8093870480911F078F5FE8
:100BC00080931F0780913F048F5F80933F04809143
:100BD00058048F5F80935804809150048F5F8093F6
:100BE0005004809151048F5F8093510420911F071E
:100BF0008091F50330E086958695869548E1849F3F
:100C0000C00111242817390714F010921F07789497
:100C1000DF91CF911F910F91FF90EF90DF90CF90D8
:100C200008955C9A88EF0E94471080913C048130BF
:100C300009F42CC1823009F014CF80914D0488232F
:100C400009F40ECF5C9A88EF0E9447100ACF80917A
:100C50003D04882309F4B7C0DD24D3941CCF813030
:100C600008F446CF843018F0853009F041CF81E098
:100C7000D81609F4A8C1E2E0DE1609F039CF809158
:100C800073048F5F8093730480912B07882309F48A
:100C900094C08091B205882309F510921F078091B6
:100CA000B605882349F480912107882329F0809193
:100CB0007C04882309F0E7C580913A06609182069A
:100CC000680F8091C6069091C7060E94402A109234
:100CD000730480917704882309F402C58091B205DA
:100CE000E091C606F091C706E80FF11D8081809360
:100CF0008E0480919B048093990480918E0480746B
:100D000080939B0480917C04882309F07FC48091A8
:100D10008E048F708F3009F4D9C480918E048F7047
:100D20008F3029F180918E040E94642A0091CC06B4
:100D3000080F10918E04107860919904802F412F34
:100D40000E94D11D112309F0C9C480E0902F935F48
:100D5000982B80914904981751F080914904809311
:100D60004A0490934904809149040E94FB0F8091AA
:100D7000EE04833009F43DC48091EE048730E9F439
:100D800080914604813009F476C580919A0590914E
:100D90009B05E091AB05F0E0EE0FFF1FE35FFD4F19
:100DA0006081718182959295907F9827807F9827A6
:100DB0000E949549862F0E944017809144048160CB
:100DC0008093440495CE52E0D52E65CE20918F04B9
:100DD000309190048091A8049091A90428173907B4
:100DE00009F4E2CD80912B07882309F0DDCD85E25F
:100DF0000E94581660918F04709190047093A9041A
:100E00006093A80485E090E00E947602CDCD8091A9
:100E100042048F5F80934204BCCDA49A85E0809306
:100E20004E048091EE048C3009F009CE8091480484
:100E300080FF0AC080912B07882309F069C2809146
:100E40005404882309F056C310924804F8CD8091C9
:100E50008604823009F0D4CD109286040E94653356
:100E6000CFCD10924304B9CD0E940E1A8091410457
:100E700080FD87CEE0914104E695F0E0E370F070EC
:100E8000EB56FB4F80810E94031A7BCE80914D046C
:100E9000882309F4E6CD88EF0E94471080913C0436
:100EA000C9CE80912B07882309F440C00E94612E8F
:100EB0001092860452CD8CE20E94642A982F809171
:100EC00073048111945F80911F07882341F48091FE
:100ED0007D04882309F454C383E20E94581680914C
:100EE0001F07843009F036CE80917D04882379F481
:100EF00080917A04823008F45EC380913E060E949D
:100F0000642A40913E06407860E00E94D11D83E251
:100F10000E9490161FCE10926B0417CE85E20E949D
:100F2000581608CE81E20E949016F4CD0E946533D7
:100F300080913C04882309F0BBCF0E948900B8CF80
:100F40008091EE04853009F464CD109287041092EC
:100F50003D041092B205109286045BCDA398B4CDE7
:100F6000883009F0C5CDF1E0DF1609F40FC382E047
:100F7000D81609F0BDCD80918D0480933E048091F8
:100F80008C0480938D040E94CB0080938C0480910C
:100F90008D048F7360E040E00E94D11D80918D042C
:100FA0000E94FB0FA5CD8091440480FFE5CD809188
:100FB00044048E7F809344040E941C178091B205E4
:100FC0000E942A17D9CD8091B6058F5F8093B60510
:100FD00080912B07882309F48BCD8091B2058F5F18
:100FE0008093B2059091B2058091F703981710F0A5
:100FF0001092B2058091B205882309F06EC08091ED
:10100000EE04833009F4A1C210E08091EE04873031
:1010100009F416C381E00E940F2A809182068F5F37
:1010200080938206C090820690918206809140064D
:10103000981708F443C080917704882319F481E05D
:10104000809384048091EE04813009F464C380911C
:10105000EE04823009F45BC382E00E940F2A1092F2
:10106000B60580917C04882369F080917A0480938E
:10107000210780912107882329F010927A0481E0CA
:101080008093B005109282068091EE04833009F4BB
:1010900095C38091EE04873009F454C380914106D2
:1010A000882309F03BC390911E078091B1059817E2
:1010B00029F080917704823008F419C48091820667
:1010C00090E082959295907F9827807F98278C5703
:1010D000994F9093C7068093C60680917C0488231D
:1010E00009F006CD8091B205E091C606F091C706E1
:1010F000E80FF11D808180938E0480918E048F70A3
:101100008F3009F4E0C280919B040E94E81D809119
:101110004A04882309F0D0C280919B04882309F0F7
:10112000E7CC80914904882309F4E2CC80914904FA
:101130000E94211010924904DBCC8091440481FF6D
:1011400016CD809144048D7F809344040E941C1727
:10115000809143040E942A170ACD0E941C176091B7
:101160008F0470919004603A710508F492C1603A5E
:10117000710509F42DC280E090E02EE030E040E0FF
:1011800050E00E946A49685E7E4F8F4F9F4F28E172
:1011900031E040E050E00E94BC49022F293008F4C1
:1011A00065C318E0812F0E942A171F5F1017D0F324
:1011B000003108F0F3CC102F812F0E9435171F5FEC
:1011C0001031D0F3EBCC0E941C178091480480FDB5
:1011D0005CC180915404882309F051C1E1E0DE161E
:1011E00009F4E0C0F2E0DF1609F082CC80917304CC
:1011F0008F5F8093730480912B07882309F478CC48
:10120000E0918206F0E0E853F94F808184FDD7C178
:1012100086E08093F5038091B205E091C606F091D7
:10122000C706E80FF11D808180938E0480919B0496
:101230008093990480918E04807480939B048091A4
:101240008E048F708F3009F4F0C180918E048F70FE
:101250008F3071F080918E040E94642A9091CC06A8
:101260006091990440918E044078890F0E94D11DAD
:1012700080914704982F92959F709093DD06982F48
:10128000977090933A06869586958695817080939F
:101290001E0780911E07882309F093C188E00E94F1
:1012A000581681E00E9490160E94101880913A060C
:1012B0008F5F0E94B01780912B07817080932B075E
:1012C00017CC81E20E94901680913F0463E00E9457
:1012D0008949992309F01ECC81E20E9458161ACC44
:1012E0000E946813882339F080918504882309F0CF
:1012F00057C10E9489000E947A13882309F428CBE1
:1013000080918504882309F423CB0E94612E20CB91
:1013100080912B07823008F497CD80915404882364
:1013200029F480919E05882309F48ECD809155047F
:1013300080934704909182069F5F909382069091DC
:1013400082069170909382066091820670E06295A9
:101350007295707F7627607F76276C57794F7093F0
:10136000C7066093C60690918206C92FD0E00E94FE
:10137000AA2CC853D94F8883E0918206F0E0E85345
:10138000F94F80818F708F5F8093F703E091820621
:10139000F0E0E853F94F808184FD00C18CE0809338
:1013A000F50352CD80912B07882309F4A1CB8091BE
:1013B000B2058F5F8093B20580915404882309F4AD
:1013C000F2C090915504809147048917D1F1F090B3
:1013D0008206F394FE220F2D10E0E801C295D2950B
:1013E000D07FDC27C07FDC27CC57D94F80915504B4
:1013F000BE010E94AA2C0853194FF8018083E09186
:101400008206F0E0E853F94F2081F801808190E0F6
:1014100030E08227932784FD14C080915504809387
:101420004704F0928206E0918206F0E0E853F94F1B
:1014300080818F708F5F8093F703D093C706C0932E
:10144000C6068091B2056091F7030E948949909386
:10145000B2058091B205E091C606F091C706E80F8B
:10146000F11D808180938E0480918E048F708F3067
:1014700009F4B7C080919B040E94E81D39CB80918C
:10148000540481500E942A17A9CE8FE00E942A1787
:10149000A0CE80E090E02EE030E040E050E00E94FE
:1014A0006A496E5070408040904028E131E040E051
:1014B00050E00E94BC49022F222309F426C110E00B
:1014C000812F0E9435171F5F1017D0F3083008F0E6
:1014D0001AC1102F812F0E942A171F5F1830D0F3D6
:1014E000103108F05BCB812F0E9435171F5F103140
:1014F000D0F354CB80915504809347040E94653308
:1015000080913C04882309F498C0809182068F5F03
:10151000809382068091820681708093820660911A
:10152000820670E062957295707F7627607F7627DD
:101530006C57794F7093C7066093C60680918206F8
:10154000C82FD0E08091470412CF80919A059091E6
:101550009B05019690939B0580939A0520919A058F
:1015600030919B058091A5059091A6052817390714
:1015700008F44ACD10929B0510929A0511E045CDD2
:10158000892F60E040E00E94D11DA6CC80E00E943F
:10159000E81D80918D040E942110AACA80E1FFCE2F
:1015A0000E946533A6CE80919E05882309F049CF1D
:1015B0000E94612E46CF80E00E94E81DA8CC88E002
:1015C00028CE88E00E94901681E00E9458166CCECA
:1015D0000E941C1787E00E942A1788E00E942A17A1
:1015E000DDCA80919B04882309F089C010929B0476
:1015F00041CF80914604813009F0BECB80919A059D
:1016000090919B0501960E940702B6CB80913A0605
:10161000609140064091B305209141060091B705C5
:10162000E090B1050E945619A2CB80918E048F7074
:1016300080938E0410929B0408CE0E94890065CF8F
:1016400080917204813009F0E5CC60911E07809191
:101650003A06409182062091CC06480F82EA95E036
:101660000E94521F8091AB0560919A0570919B0575
:101670004091A2050E94B81F80919A0590919B0508
:10168000019690939B0580939A05E091AB0520917C
:101690009A0530919B05F0E0EE0FFF1FE35FFD4FD1
:1016A000808191812817390708F4B4CC1092720414
:1016B00083E20E949016AECC80914A040E942110D1
:1016C00010924A0429CD10929B041DCD80918E0466
:1016D0008F7080938E0410929B041FCB80E836CBD2
:1016E00080913A06609140064091B30520914106F1
:1016F0000091B705E090B1050E945619EFCA81E04C
:101700000E94E81D73CF102FEBCE10E0E3CE81E0F6
:1017100080938404A1CC8093840499CC0E94FC29FA
:1017200080917704823008F0C9CC8091DD06609109
:101730001E0740913A062091400604E816E00E94F8
:10174000072DBCCC80917204813009F0A7CC809128
:101750009E058823B9F01092720410929E05809124
:10176000AB0560919A0570919B050E948F1F809137
:10177000AB050E941B209093A6058093A50583E2EC
:101780000E94901680919F05882309F487CC1092BF
:101790009F058091AB0560919A0570919B056C192E
:1017A0000E947F1F8091AB050E9412209093AD058F
:1017B0008093AC0580E00E94901670CC80919E05CD
:1017C000882309F089C080919F05882309F450C0BF
:1017D00010929B0510929A058091E9048093AB05C5
:1017E0008091AB050E941B209093A6058093A505D0
:1017F0008091AB050E9412209093AD058093AC05BB
:101800002091AC053091AD058091A5059091A6057C
:101810002817390720F01092AD051092AC05809181
:101820009F05882309F04AC08091AB0560919A0515
:1018300070919B050E946C208093A2058091AB055E
:101840006091A20549EF55E021EB35E003EB15E08F
:1018500095ECE92E96E0F92E0E94321F81E08093EC
:1018600041068091C5068093CC0613CC18E0A4CC29
:101870001123A9F2ADCF80919A0590919B05019615
:101880000E94070282CA81E00E94E81D80E00E9457
:10189000E81D6091400684E896E04EED56E028EBA6
:1018A00035E00E946F2B10927C048AE00E94802A0F
:1018B00010929B0482E00E943C0FFEC910929F058B
:1018C0008091AC059091AD0590939B0580939A050E
:1018D00080E00E949016A8CF10929E0510929B0562
:1018E00010929A0583E20E94901611E06CCF8091CD
:1018F000B10580931E0719CF07C080914C04815019
:1019000080934C040E949A0480914C048823A9F788
:101910000895AF92BF92CF92DF92EF92FF920F9312
:101920001F93DF93CF93CDB7DEB760970FB6F894D0
:10193000DEBF0FBECDBF0E9487020E942A038091A6
:101940006E00826080936E0083E084BD85BD8AEF67
:1019500087BD84E896E09093C7068093C606F99900
:10196000FECF82E090E092BD81BDF89A80B5982FBD
:10197000937090933C048295817080937D04F999D3
:10198000FECF87E090E092BD81BDF89A80B58823B4
:1019900011F0813208F080E180930002F999FECFC6
:1019A00083E090E092BD81BDF89A80B58F708093FE
:1019B000C604F999FECF84E090E092BD81BDF89A0B
:1019C00080B58F708093B30488E090E00E9451024C
:1019D0008093A20420918F0430919004280F391F26
:1019E000309394042093930485EB9BE39093AC0491
:1019F0008093AB0483E393E19093B2048093B104AA
:101A000085E694ED9093A7048093A6040E94FC00C1
:101A10000E94FC000E94FC00BC0188E090E00E9453
:101A20007602F999FECF8AE090E092BD81BDF89AE6
:101A300090B5892F8F708093AD048091AD04833071
:101A400010F01092AD0492959F709F5F9093B00438
:101A50008091B004823018F482E08093B004F99948
:101A6000FECF8DE090E092BD81BDF89A60B5862FE3
:101A70008C59893C08F42AC160ED72E183E190E061
:101A8000F8946093090270930A0280930B0290937A
:101A90000C02F999FECF8EE090E092BD81BDF89ADC
:101AA00040B5493008F409C142E08CE08093AA04B3
:101AB0004093A3040E94032E789400E010E01DC020
:101AC0008091F3040E942A170E946718C801849627
:101AD00068E270E00E94A9490E94FD190E949016D8
:101AE00080E10E943C0FC80187709070892B69F0DB
:101AF0000F5F1F4F0C32110579F0083208F7802F65
:101B00000E94FD190E945816DBCF0E94A6150F5F98
:101B10001F4F0C32110589F70E9407170E946718A2
:101B20000E94A61580E00E94E113882331F083E033
:101B30000E94E113882309F022C183E00E94E1138F
:101B4000882309F0D3C08091F3048093DD061092BE
:101B50001E071092B10510923A0681E0809340066C
:101B6000109241068091DD0660911E0740913A0671
:101B70002091400604E816E00E94072D60913A0685
:101B8000C8010E94402A0E94CB290E94A61580917C
:101B90004404836080934404109245048091EE04D1
:101BA000873009F487C08830B0F5823009F45EC010
:101BB000833008F045C0882309F452C0813009F40D
:101BC00052C00E94A61580914C04882359F0809140
:101BD0004C04815080934C040E949A0480914C04E0
:101BE0008823A9F70E94CB29882379F68091EE04F7
:101BF000863039F781E00E940D14882311F380E0CC
:101C00000E94E1138823E9F20E9407170E946718D7
:101C1000E0E0F0EF19948C3009F449C08D3038F4CD
:101C2000883069F18B3069F60E944E23AECF8E303A
:101C300019F18E30F0F08F3021F60E94A22EA5CF40
:101C4000843059F0843030F0853009F0BACF0E94EA
:101C50004C359BCF0E94E32598CF0E94F01D95CF75
:101C60000E946D1292CF0E94A4418FCF0E94853FA7
:101C70008CCF0E94364889CF0E94501A86CF0E948E
:101C800007170E94A61580914C04882359F0809173
:101C90004C04815080934C040E949A0480914C041F
:101CA0008823A9F70E94CB29882359F36ECF0E947D
:101CB000E7106BCF0E949C2768CF242F30E0C9012A
:101CC000880F991F820F931F880FF0CE772767FD2B
:101CD0007095872F972F22EE34E040E050E00E946D
:101CE0006A4960537D4E8C4E9F4FCACE8CE00E9455
:101CF000E113882309F427CF6E010894C11CD11C7D
:101D0000FF24B1E1AB2EB12CAC0EBD1EAFE0EA2E2C
:101D100086010E94FC00F801908381830E5F1F4FB3
:101D20000A151B05B1F7F60104C03196E017F1075B
:101D300089F02081822F90E08F7090700D9724F0B1
:101D4000822F8F708083282F2D3079F78E2F8C195A
:101D50008F3099F480E060E04F2D21E086010E94F1
:101D60007C2D85E50E941C1A0E946718F394F0E808
:101D7000FF1671F60E940717E6CEE082D6CF1092CA
:101D80003C0410927D0460917D0470E0617070707D
:101D900062957295707F7627607F762782E090E06B
:101DA0000E946C020E94032E1092C6041092B3048B
:101DB00083E090E060E00E946C0284E090E060913B
:101DC000B3040E946C0288E790E0909390048093A3
:101DD0008F0485E090E068E770E00E94760280E181
:101DE000809300026091000287E090E00E946C0204
:101DF0001092AD0488E08093B0048091B0046091AB
:101E0000AD0490E0019782959295907F9827807F0E
:101E10009827682B8AE090E00E946C028DE090E0A9
:101E200060E00E946C02F89480ED92E1A3E1B0E0E2
:101E30008093090290930A02A0930B02B0930C02C4
:101E400078948CE08093AA0482E08093A3048EE0CF
:101E500090E062E00E946C0210E082E20E94C416F0
:101E600083E20E94C4160E94671882E30E943C0F1E
:101E70001F5F183291F77ECF20EA3FE0E22FF32F69
:101E80003197F1F78A95D1F70895882309F41EC098
:101E90009AEF20EA3FE0E22FF32F3197F1F79A957E
:101EA000D1F7E22FF32F3197F1F79A95D1F7E22F7F
:101EB000F32F3197F1F79A95D1F7E22FF32F31975E
:101EC000F1F79A95D1F7815009F0E5CF0895109276
:101ED000BC041092C50408951F93CF93DF93EC01C7
:101EE000142F6F777885772309F44CC0462F50E084
:101EF000888190E08F7790704817590779F121E039
:101F000030E00DC0D901FE01E20FF31F808190E0A7
:101F10008F7790702F5F3F4F8417950709F1271730
:101F200088F3272F2F5F293030F128E0822F922F5E
:101F30009150FE01E80FF11DDE01A90FB11D8C913A
:101F40008083892F9923A1F71536C0F480E0862B72
:101F500088832887DF91CF911F910895A0E0B0E09A
:101F6000153670F480E0AC0FBD1F862B8C93DF918B
:101F7000CF911F9108952223C9F6E6CF80E8E7CFDD
:101F800080E8F1CF81E091E021E0D2CFCF93DF93E1
:101F9000EC0138853323B9F06F7770E0888190E0E9
:101FA0008F7790706817790789F0FE0120E008C0EC
:101FB000818190E08F77907031966817790739F0BA
:101FC0002F5F2317A8F3DF91CF91089520E03230DF
:101FD00068F0922F9F5FFE01E20FF11DDE01A90F55
:101FE000B11D8C918083292F9317A0F3315038872E
:101FF000DF91CF910895282F9091B3048091C00074
:1020000085FFFCCF90699093C6008091C00085FF4A
:10201000FCCF822F8F778093C60027FD09C0909157
:102020002F028091C00085FFFCCF9093C6000895D9
:1020300090912D028091C00085FFFCCF9093C60047
:102040000895282F9091B3048091C00085FFFCCFA4
:1020500090689093C6008091C00085FFFCCF822FCE
:102060008F778093C60027FD09C090912F02809141
:10207000C00085FFFCCF9093C600089590912D027B
:102080008091C00085FFFCCF9093C6000895982FE3
:102090008091C00085FFFCCF9093C60080E090E067
:1020A0000895909156048091570420E030E09817ED
:1020B00011F021E030E0C90108959091560480911B
:1020C00057049817D1F3F89490915604E92FF0E053
:1020D000E953FB4F80819F5F909356049091560483
:1020E0009F7190935604789490E0089590915604CF
:1020F00080915704981729F00E945D10482F87FDA2
:1021000003C040E0842F0895582F52955F705F30D0
:10211000C9F3282F30E02F7030708091C60490E012
:102120002817390771F750935304ECCF9091B304FB
:102130008091C00085FFFCCF906B9093C60080918A
:10214000C00085FFFCCF8BE78093C6008091C00064
:1021500085FFFCCF1092C600089580913C04823028
:1021600049F08091C00085FFFCCF8CEF8093C600C2
:102170000E949610089590913E048913089580E07E
:102180000E94E81D8FEF80933E0408951F93182F3F
:10219000962F6623B9F060E080913E048F3F09F0EE
:1021A00061E0953648F4812F895140E00E94D11DAD
:1021B00010933E041F910895812F895141E00E94A0
:1021C000D11DF6CF60E00E94BB101F910895FF92D1
:1021D0000F931F9380919E05817080939E0580913F
:1021E0009E05809385040E94071780919E05882391
:1021F00009F032C10E9467188BE090E00E946502EE
:10220000809330028CE090E00E946502809331025E
:10221000FF2410E00E94A6150E947C0C0E94CB298E
:10222000882309F04AC0909156048091570498176A
:1022300069F00E945D10682F87FD6DC08091530486
:10224000883009F4AEC0893009F479C0112371F4E3
:102250002091BC04222349F48091C504882329F4E9
:1022600080912B07882309F4E2C010E087E10E94E7
:102270003614882379F280919E058F5F80939E05A6
:1022800080919E05817080939E0580919E0580932C
:10229000850480E00E94901680919E05882309F4B1
:1022A000B9CF80E00E9458160E94A6150E947C0CAF
:1022B0000E94CB29882309F4B6CF0E94961081E0B2
:1022C0008093400680911E078093B10510924106CD
:1022D0008091DD0660911E0740913A0620914006EC
:1022E00004E816E00E94072D60913A06C8010E949A
:1022F000402AFF2061F08BE090E0609130020E9464
:102300006C028CE090E0609131020E946C021F919F
:102310000F91FF900895482F42954F704F3009F468
:1023200098C0282F30E02F7030708091C60490E064
:102330002817390709F48DC0109253046BCF67FD3D
:10234000BAC0062F0E945D10482F112309F08ECFCE
:1023500050913002051748F0852F90E00F96202FFE
:1023600030E0821793070CF082C0509131020517BC
:1023700008F46ECF852F90E00C96202F30E0821766
:1023800093070CF465CF051B8DEB94E0602F0E9442
:102390006C0F8091BD048F778093CC062091BC0494
:1023A00059CF67FD84C0062F0E945D10112371F57F
:1023B00040913002041748F0842F90E00F96202FB0
:1023C00030E0821793070CF06BC040913102041784
:1023D00008F43ECF842F90E00C96202F30E0821737
:1023E00093070CF435CF041B8DEB94E0602F0E9413
:1023F000C60F8091C504882309F42ACF8091BD04BB
:102400008F778093CC062091BC0424CF113009F43F
:1024100056C089E10E9490160093310280919E057A
:10242000809385042091BC04FF24F39413CF84E0AF
:102430000E9436148823A1F485E00E943614882374
:1024400009F413CF1092850489E10E94581612E016
:102450000DCF40935304F2CE80E00E945816CACEAE
:102460001092850480E20E94581611E0FFCE051BF1
:1024700084EB94E0602F0E946C0F2091BC042093A9
:1024800054048091B4048F77809355048091F304B1
:10249000909155048295807F890F80935504DACE00
:1024A000041B84EB94E0602F0E94C60FE6CF0E94CD
:1024B0005D10082F79CF0E945D10082F43CF80E276
:1024C0000E9490160093300280919E0580938504AF
:1024D0002091BC04FF24F394BDCE1F930E941C17CF
:1024E0008091C6040E942A170E94A61584E60E94C5
:1024F0003C0F0E94A61584E60E943C0F0E94A61580
:102500008FEF80933E040E94A6150E947C0C0E94CF
:10251000CB29882311F59091560480915704981780
:1025200091F30E945D10482F87FD1BC080915304DA
:10253000883049F1893039F747FD32C0142F0E94A5
:102540005D10682F812F0E94C6100E94A6150E9460
:102550007C0C0E94CB298823F1F20E9496101F91D7
:102560000895582F52955F705F30B9F0282F30E0F2
:102570002F7030708091C60490E02817390769F0F9
:1025800010925304C0CF47FD0FC0142F0E945D105E
:10259000682F812F0E94BB10B6CF50935304C6CF33
:1025A0000E945D10182FCBCF0E945D10182FEECF28
:1025B0001F920F920FB60F920BB60F9211242F930A
:1025C0003F934F935F936F937F938F939F93AF93BB
:1025D000BF93EF93FF939091C6009A3F09F442C0D6
:1025E0009C3FA9F1983F09F44AC080915704E82F15
:1025F000F0E0E953FB4F90838F5F80935704809105
:1026000057048F718093570490915704809156041A
:10261000981751F4809156048F5F809356048091EF
:1026200056048F7180935604FF91EF91BF91AF9143
:102630009F918F917F916F915F914F913F912F91DA
:102640000F900BBE0F900FBE0F901F9018958091AA
:102650008504882349F380913C04823029F70E9445
:10266000612EE2CF80913C048230F1F680918504A6
:10267000882311F00E9465330E948900D5CF809194
:102680008A0490918B0490933A04809339041092B9
:102690008B0410928A0480913C04823029F6809148
:1026A000390490913A049695879590935A048093B3
:1026B000590481E080934D0480914C048F5F809396
:1026C0004C04B2CF80913C04813009F05F980895AA
:1026D00099B1991F9927991F80915B04882311F460
:1026E000992321F490935B0480E0089590935B0418
:1026F00081E0089599B1991F9927991F80915C04F1
:10270000882311F0992321F090935C0480E00895D0
:1027100010925C0481E008958AB1806F8AB98BB110
:102720008F708BB908958AB18F708AB98BB18F7011
:102730008BB9089580913C04882321F45C9881E052
:102740000E943C0F5F9A0895AC01F894289800000D
:10275000000000000000289A20E030E01EBC0DB40C
:1027600007FEFDCF8EB5FA01E20FF31F80832F5FC6
:102770003F4F2330310591F77894089516980895C6
:10278000169A089520B1269526952F70822F90E0F5
:102790002695322F369536952270322B880F991F49
:1027A000282F2470322B880F991F880F991F88704B
:1027B000382B8FE0831B089580B1869586958F70A6
:1027C0000895282F883188F4E82FE695E695E69558
:1027D000F0E0EC50FB4F808190E0277002C09595AF
:1027E00087952A95E2F78170089580E00895282F53
:1027F000883188F4E82FE695E695E695F0E0E55116
:10280000FB4F808190E0277002C0959587952A95AF
:10281000E2F78170089580E00895282F883188F4C8
:10282000E82FE695E695E695F0E0E151FB4F8081D3
:1028300090E0277002C0959587952A95E2F7817000
:10284000089580E008958091F404882321F4809114
:10285000F504882319F090E0892F089590E0809185
:10286000F6048823C9F791E0892F0895282F88312D
:10287000A0F4482F469546954695277081E090E054
:10288000382F01C0330F2A95EAF7A42FB0E0FD01DD
:10289000E551FB4F8081832319F420E0822F0895B6
:1028A000232F30E020953095AC50BB4F8C9190E0B9
:1028B00028233923232B89F7342F3F5F832F63E0AD
:1028C0000E948949E92FF0E0EC50FB4F808188237A
:1028D00021F720E0832F8F5F0E948949E92FF0E0E4
:1028E000EC50FB4F80818823C9F621E0D7CF1F939E
:1028F000CF93DF93C4E4D2E010E088810E94E1131B
:10290000882329F41F5F21961D30B9F71FEF812F0F
:10291000DF91CF911F9108951F93CF93DF93C4E46C
:10292000D2E010E088810E94F713882349F41F5FEA
:1029300021961D30B9F780E0DF91CF911F91089566
:10294000812F8F5FDF91CF911F9108951F93CF93B8
:10295000DF93C4E4D2E010E088810E940D14882344
:1029600049F41F5F21961D30B9F780E0DF91CF91C8
:102970001F910895812F8F5FDF91CF911F9108954F
:102980001F93CF93DF93CCE3D2E010E088810E94C5
:10299000E113882349F41F5F21961830B9F780E0CE
:1029A000DF91CF911F910895812F8F5FDF91CF919C
:1029B0001F9108951F93CF93DF93CCE3D2E010E0F3
:1029C00088810E94F713882349F41F5F21961830ED
:1029D000B9F780E0DF91CF911F910895812F8F5F2C
:1029E000DF91CF911F9108951F93CF93DF93CCE395
:1029F000D2E010E088810E940D14882349F41F5F03
:102A000021961830B9F780E0DF91CF911F9108959A
:102A1000812F8F5FDF91CF911F910895CF93DF9327
:102A2000CCE3D2E088810E94E113882349F4219607
:102A300082E0C434D807B1F780E0DF91CF910895E8
:102A400081E0DF91CF910895FF920F931F93CF9371
:102A5000DF93CCE3D2E0FF2400E006C00F5F2196B5
:102A600082E0C434D80789F01881812F0E94E113D5
:102A70008823A1F7812F0E940D14882381F3F394FA
:102A8000219682E0C434D80779F781E0F81639F04E
:102A900080E0DF91CF911F910F91FF90089580E02A
:102AA0000730B9F781E0F5CF1F93CF93DF93C2E3EF
:102AB000D2E010E088810E94F713882349F41F5F59
:102AC00021961A30B9F780E0DF91CF911F910895D8
:102AD000812F8F5FDF91CF911F91089580915E04C8
:102AE00010925E04089580E00895382F883100F533
:102AF000282F277081E090E0982F01C0990F2A9528
:102B0000EAF7832F869586958695A82FB0E0FD017C
:102B1000E551FB4F8081892369F4FD01E151FB4FB1
:102B20008081892371F4AC50BB4F8C91982339F488
:102B300080E00895832F0E94361982E0089583E093
:102B40000895832F0E943E1981E00895EF92FF922D
:102B50000F931F93DF93CF9300D000D0CDB7DEB794
:102B60001092EB041092EF041092EC041092F00417
:102B70001092ED041092F10480915F048A3068F4A1
:102B800026960FB6F894DEBF0FBECDBFCF91DF9172
:102B90001F910F91FF90EF90089510925F04169887
:102BA0007E010894E11CF11CC7010E94A4138091CE
:102BB000F4048C838091F5048D838091F6048E83D8
:102BC00060E070E001E010E0E62FE695E695E6951E
:102BD000F0E0CB0187709070980102C0220F331F84
:102BE0008A95E2F7C901AF014C505B4FD701AE0F98
:102BF000BF1F3C91E950FB4F2081232B2823809558
:102C0000FA0130818323282B20836F5F7F4F683147
:102C10007105D1F60E94C213982F96959093F304F4
:102C20008093E904169A40E050E0BE016C5F7F4F4C
:102C3000DA01A950BB4FF701E40FF51F80818C9397
:102C4000FB01E40FF51F2081FA01EC50FB4F90814E
:102C5000FA01E551FB4F822F809589238083FA0189
:102C6000E151FB4F9095922390834F5F5F4F43302C
:102C70005105F1F690B1969596959F708091E70475
:102C8000891721F0109260049093E704809160040A
:102C90008F3630F09093E8048091E8048093E70445
:102CA00082E00E94E11380934B040E94671868CF72
:102CB000282F8832C0F4E82FE695E695E695F0E0F7
:102CC000277081E090E001C0880F2A95EAF7DF01C4
:102CD000AF59BB4F2C91282B2C93EA59FB4F809571
:102CE0002081822380830895282F8832C0F4E82F22
:102CF000E695E695E695F0E0277081E090E001C06A
:102D0000880F2A95EAF7DF01AA59BB4F2C91282B8F
:102D10002C93EF59FB4F8095208182238083089567
:102D2000282F8832C8F4E82FE695E695E695F0E07E
:102D3000277081E090E002C0880F991F2A95E2F782
:102D40008095DF01AF59BB4F2C9128232C93EA5972
:102D5000FB4F2081822380830895282F883298F4A6
:102D6000E82FE695E695E695F0E0EA59FB4F2770E7
:102D700081E090E002C0880F991F2A95E2F78095C4
:102D80002081822380830895282F883290F4E82FB1
:102D9000E695E695E695F0E0EF59FB4F277081E068
:102DA00090E002C0880F991F2A95E2F7208128271A
:102DB00020830895E82F883298F4282F277081E027
:102DC00090E002C0880F991F2A95E2F7E695E695F4
:102DD000E695F0E0EA59FB4F20812823822F0895E1
:102DE00020E0822F0895982F969596959695E1E686
:102DF000F4E0E90FF11D208130E0877002C03595C5
:102E000027958A95E2F721703070C90108951092D4
:102E1000650410926404109263041092620410928C
:102E2000610410926A04109269041092680410926E
:102E30006704109266040895CF93DF93C0EBD2E04D
:102E400089910E94901682E0C03CD807C9F7DF91B3
:102E5000CF910895803108F00895E82FF0E0E05513
:102E6000FD4F80810E9458160895803108F0089522
:102E7000E82FF0E0E055FD4F80810E949016089504
:102E80000F931F93CF93DF93082FC0EBD2E010E096
:102E900007C088810E9458161F5F2196103149F0A3
:102EA0001017B8F388810E9490161F5F2196103189
:102EB000B9F7DF91CF911F910F910895803108F0FC
:102EC0000895E82FF0E0E055FD4F80810E947416D0
:102ED0000895803110F080E00895E82FF0E0E0558B
:102EE000FD4F80810E94F3160895803110F080E03C
:102EF0000895E82FF0E0E055FD4F80810E94DA163A
:102F00000895883108F00895E82FF0E0E557FD4F67
:102F100080810E9458160895883108F00895E82F9E
:102F2000F0E0E557FD4F80810E94741608958831C6
:102F300008F00895E82FF0E0E557FD4F80810E94EA
:102F400090160895CF93DF93CBE8D2E089910E9449
:102F5000901682E0C33AD807C9F7DF91CF91089560
:102F6000E82F8150883008F00895F0E0EE57FD4FCB
:102F700080810E94581608950F931F93CF93DF937B
:102F8000082FC3E8D2E011E007C088810E949016A4
:102F90001F5F2196193069F01017B9F7E12FF0E0A3
:102FA000EE57FD4F80810E9458161F5F2196193001
:102FB00099F7DF91CF911F910F910895E82F8150DC
:102FC000883008F00895F0E0EE57FD4F80810E94B0
:102FD00090160895E82F8150883008F00895F0E0A9
:102FE000EE57FD4F80810E9474160895E82F81509E
:102FF000883010F080E00895F0E0EE57FD4F8081BA
:103000000E94DA160895E82F8150883010F080E091
:103010000895F0E0EE57FD4F80810E94F316089569
:10302000CF93DF93C3E8D2E089910E94901682E0AB
:10303000CB38D807C9F7DF91CF9108958D3008F0CC
:103040000895E82FF0E0ED55FD4F80810E9458165D
:1030500008958D3008F00895E82FF0E0ED55FD4F0C
:1030600080810E94901608958D3008F00895E82F11
:10307000F0E0ED55FD4F80810E9474160895E3EA5B
:10308000F2E0E80FF11D80810E94DA160895CF93D7
:10309000DF93C3EAD2E089910E94901682E0C03BA0
:1030A000D807C9F7DF91CF9108950E94471884E0AF
:1030B0000E94901683E00E94901688E00E9490166D
:1030C00081E00E94901682E00E9490160895F89484
:1030D000179820E030E090916B04F901EA59FB4F1A
:1030E00080819823F901EF59FB4F8081982B9EBD79
:1030F0000DB407FEFDCF2F5F3F4F2530310559F747
:10310000179A78940895E1E6F4E0A6E6B4E08081A9
:103110009D91892B819384E0E636F807C1F70895E5
:10312000E1E6F4E0A6E6B4E09D91909580818923E4
:10313000819384E0E636F807B9F70895E1E6F4E014
:10314000A6E6B4E020819C91892F822319F0909506
:10315000922390831D92319684E0E636F80791F72A
:1031600008951F93182F84E00E949016123049F0A2
:1031700083E00E949016113071F01F3F39F01F91CB
:10318000089583E00E9474161F91089584E00E94C0
:1031900058161F91089583E00E9458161F910895B4
:1031A0000F931F93CF93DF93182F87FD50C086E1B5
:1031B0000E949717812F829586958695837080FF50
:1031C00029C085E10E9481171F7349F11731A0F5CD
:1031D0008FEF0E94B11884E10E949717012F10E031
:1031E000CBE0D0E0C017D10731F0FE01E856FD4F2B
:1031F00080810E9490162196C831D10599F7085612
:103200001D4FF80180810E945816DF91CF911F91C8
:103210000F91089585E10E9497171F73B9F680E01A
:103220000E94B1180E94471884E10E948117DF9123
:10323000CF911F910F910895143268F0103370F4FC
:10324000185181E00E94B118112329F6EBCF86E1D5
:103250000E948117AFCF1C5080E0F4CF1C3318F4CC
:10326000145282E0EFCF105383E0ECCFEBE8F2E0B2
:10327000E80FF11D80810E9458160895EBE8F2E0F6
:10328000E80FF11D80810E9490160895E3E8F2E0B6
:10329000E80FF11D80810E9458160895E3E8F2E0DE
:1032A000E80FF11D80810E9490160895DF92EF9241
:1032B000FF920F931F93CF93DF93F02EDE2C2223E8
:1032C00071F1022F040FE42EC3E8D2E010E00BC02E
:1032D000101758F41F15D9F088810E9458161F5FE7
:1032E0002196183049F01E1598F788810E94901693
:1032F0001F5F21961830B9F781E08D15A0F4DF919A
:10330000CF911F910F91FF90EF90DF900895E12FE3
:10331000F0E0ED57FD4F80810E947416E0CF062F3C
:10332000080FE82ED1CFDD2071F088E00E949016C2
:1033300081E00E945816DF91CF911F910F91FF906D
:10334000EF90DF90089588E00E94581681E00E9477
:103350009016DF91CF911F910F91FF90EF90DF902A
:103360000895FF920F931F93082FF62E84E00E947A
:10337000901683E00E94901688E00E94901681E0EB
:103380000E949016102F04FD34C015FD29C007FDC2
:103390002CC016FD21C00E944718FF2099F0802FF5
:1033A0008F708D3098F08BE10E9458168CE10E944E
:1033B00058168FE00E9458168EE00E9458168DE035
:1033C0000E9458161F910F91FF9008950E941E1899
:1033D0001F910F91FF90089581E00E945816DBCF56
:1033E00083E00E94581607FFD4CF88E00E94581649
:1033F000D0CF84E00E945816C8CFE1E5F2E0E80F94
:10340000F11D808108958A3008F00895E82FF0E0DA
:10341000E758FD4F80810E9458160895CF93DF939F
:10342000C9E7D2E089910E94901682E0C338D8079C
:10343000C9F7DF91CF9108959091610498279093F7
:1034400061049091620498279093620490916304C0
:103450009827909363049091640498279093640450
:10346000909165049827909365040895AC016115C7
:103470007105A1F020E0E0E0A0E0B0E0A40FB51FEE
:103480008C91E827F0E0E853FD4FE0812F5FA22FF9
:10349000B0E0A617B70790F38E2F0895E0E0FCCFB9
:1034A0000E94A6150E947C0C0E94CB298823C1F3A0
:1034B0000895EF92FF920F931F93CF93DF937C01B8
:1034C0008B016115710561F0C0E0D0E0F701EC0FF0
:1034D000FD1F80810E94EA012196C017D107B0F339
:1034E000DF91CF911F910F91FF90EF90089522E40B
:1034F0002093FA041092FB0422E02093FC049093A2
:10350000FD048093FE04AAEFB4E0E0E08D91E8278B
:10351000F0E0E853FD4FE08184E0AF3FB807B1F73A
:10352000EC93CD01059766E070E00E94591A08956A
:1035300090E89093FA041092FB0421E02093FC049D
:103540008093FD04A8ECB2E090914803FD01E90FDF
:10355000F11D90819227FD01E90FF11D90819827BF
:10356000A90FB11D8C918093FE048AEF94E065E071
:1035700070E00E94591A08951F920F920FB60F9291
:103580000BB60F921124DF92EF92FF920F931F93CD
:103590002F933F934F935F936F937F938F939F935B
:1035A000AF93BF93CF93DF93EF93FF931091CE0030
:1035B0008091C702882309F46EC080916E049091B7
:1035C0006F04895E934008F080C080916C04803461
:1035D00008F089C0282F2F5FE82FF0E0E65CFA4F53
:1035E000108320936C0410926F0410926E042330A9
:1035F00008F451C070913A0590913B0580E06091CC
:103600003C05462F50E0482B592B30E0CA01049668
:103610002817390708F43FC09A012D5F3F4FF90181
:10362000E65CFA4F10812115310509F401C190E0E3
:10363000E0E0A0E0B0E0A65CBA4F8C91E827F0E0B3
:10364000E853FD4FE0819F5FA92FB0E0A217B307B9
:1036500090F31E1709F450C02115310509F4EAC092
:1036600090E0E0E0A0E0B0E0A65CBA4F8C91E827E3
:10367000F0E0E853FD4FE0819F5FA92FB0E0A21773
:10368000B30790F38E2F90E00E94C60110926C0455
:1036900080E00E94981AFF91EF91DF91CF91BF9146
:1036A000AF919F918F917F916F915F914F913F91DA
:1036B0002F911F910F91FF90EF90DF900F900BBE15
:1036C0000F900FBE0F901F9018950E941C170E941C
:1036D000671810933A0581E080936C0410926F0490
:1036E00010926E04D8CF0E94981A10926C04109217
:1036F0006F0410926E04CFCF713809F492C1723802
:10370000B0F5713109F42BC1723108F096C07130F7
:1037100051F1703131F080E00E94981A10926C04DF
:10372000BACF6231C1F780913D05082F10E0000F3C
:10373000111F000F111F000F111F80913E05080F70
:10374000111D02951295107F1027007F1027CFE3DF
:10375000D5E08991B8010E94B31E0F5F1F4F85E02D
:10376000CF34D807B1F781E00E94981AD7CF7638C6
:1037700009F435C1773808F073C0723809F484C190
:10378000753849F64330510509F0A5C030913D0523
:10379000932F80E020913E05E22EFF24E82AF92AAB
:1037A000D0903F05EAE3ED1508F4B6CF7093FA0424
:1037B0001092FB04F2E0DF0ED092FC048EEFD80EE4
:1037C0003093FD042093FE04DD2071F00FEF14E030
:1037D000E701CE010E94F71EF80181938F01219627
:1037E0009E012E192D15A8F38091FC04682F6D5FA2
:1037F00009F4D5C1AAEFB4E090E08E5F282F30E045
:1038000025503B4F8D919827E92FF0E0E853FD4F6D
:103810009081A217B307B1F7E62FF0E0E650FB4F17
:1038200090836F5F8AEF94E070E00E94591A76CF20
:10383000E0E00FCF80E090E027CF703409F453C16F
:10384000713409F068CF623009F065CF90913D0581
:1038500080E020913E05820F911D0E94D2025ECF32
:103860007738E9F1783809F056CF7093FA0410925E
:10387000FB0480913D05813009F46AC1813008F074
:103880005BC180E18093FD041092FE048093FF04ED
:103890001092000584E047E0A7E0B0E068E070E047
:1038A0008093FC0490E020E030E0F901E650FB4F0B
:1038B00080819827E92FF0E0E853FD4F90812F5F3A
:1038C0003F4F241790F3A650BB4F9C938AEF94E090
:1038D0000E94591A23CF80E00E94981A1FCF80912E
:1038E0003D05882309F006C14230510509F014CF87
:1038F000E0913E05E43008F00ECF89E18093FA04B0
:103900001092FB0480E18093FC042E2F30E022957E
:103910003295307F3227207F3227ADEFB4E0F901B6
:10392000EC57F94F80818D932F5F3F4F85E0AD308D
:10393000B807A9F75397E0E08D91E827F0E0E85346
:10394000FD4FE081F5E0AD30BF07B1F7E0930D0525
:10395000CD01439764E170E00E94591ADFCE6230D6
:1039600009F0D9CE80913D05082F10E0000F111FFE
:10397000000F111F000F111F80913E05080F111D30
:1039800002951295107F1027007F102789E1809300
:10399000FA041092FB0480E18093FC04CDEFD4E0A4
:1039A000C8010E94F71E89930F5F1F4F35E0CD308D
:1039B000D307B1F7DE015397E0E08D91E827F0E0FF
:1039C000E853FD4FE081CA17DB07B9F7E0930D0517
:1039D0008AEF94E064E170E00E94591A9FCE9091C2
:1039E0003D0580E020913E05E22EFF24E82AF92AD9
:1039F0002EEFD22ED60E63506A3308F06CCFDD2046
:103A000009F4B1CE0FE315E0E701F80181918F01D0
:103A1000BE010E94B31E21969E012E192D15A8F3FA
:103A2000A2CE87E190E09093FE048093FD048EEC9B
:103A300090E0909300058093FF04E0ECF2E0A1E0B9
:103A4000B5E081918D9322E0E63CF207D1F781E861
:103A50008093FA041092FB048AE08093FC04AAEF9E
:103A6000B4E0E0E08D91E827F0E0E853FD4FE0811D
:103A700035E0A730B307B1F7EC93CD010D976EE0B9
:103A800070E00E94591A4ACE4230510509F023CF06
:103A900030913D05332309F468C090913E0520E044
:103AA00082E88093FA041092FB0483E08093FC0484
:103AB0003093FD049093FE042093FF04AAEFB4E03A
:103AC000E0E08D91E827F0E0E853FD4FE08185E0EC
:103AD000A030B807B1F7EC93CD01069767E070E02E
:103AE0000E94591A1BCE80918F04909190040E94DD
:103AF000771A14CE813009F00ECE4231510509F00B
:103B00000ACEE0913E05E43008F005CE2E2F30E0DD
:103B1000AFE3B5E022953295307F3227207F322700
:103B20008D91F901EC57F94F80832F5F3F4F85E06E
:103B3000AF34B807A9F717CE883009F0ECCD81E093
:103B40008093FD0444E0A4E0B0E065E070E0A8CE1E
:103B500088E08093FD0480E18093FE0482E045E0EC
:103B6000A5E0B0E066E070E09BCE90913E0597380E
:103B700060F4953870F4993181F0993120F0892FF3
:103B80008158823030F020E08BCF973821F0983880
:103B9000D1F721E085CF24E083CF20E181CF90E0F1
:103BA0003BCE2C98803408F08FE3611160E444230D
:103BB00049F090E0882349F0682B962B98B92C9A0D
:103BC0002D9A089590E88823B9F7962B98B908950F
:103BD000882319F42D982C980895469A2C980895C6
:103BE0009F92AF92BF92CF92DF92EF92FF920F938C
:103BF0001F93CF93DF930E941C178091B3040E9400
:103C00002A170E94A6150E946E15BB249924AA2487
:103C1000CC240E94A6150E947C0C0E94CB298823EC
:103C200009F075C02B2D3CE02302C001112497E15F
:103C3000D92ED80EEA2CE294EE0CEE0C80ECE822A1
:103C4000C0E0D0E009C0802F0E940D14882319F530
:103C50002196CD30D10559F1FC2EFE01E853FC4FE1
:103C60000081802F0E94F713882369F31C2F1D0DFC
:103C7000812F6C2D4A2D0E94D11D812F8E290E94EB
:103C8000FB0F8C2F0E941E18CC24C394802F0E94FF
:103C90000D148823E9F28F2D8D0D8E290E9421109D
:103CA0008F2D0E9429182196CD30D105A9F68FE0DD
:103CB0000E94F713882309F444C081E08B150CF0AF
:103CC00050C09B1429F08B2D0E94B1180E946718D8
:103CD00084E10E94F713882351F080E0AA2009F4C0
:103CE00081E0A82E8823C9F188E00E94581686B189
:103CF00090E08F739070892BC1F49B2C0E94A615C5
:103D00000E947C0C0E94CB29882309F48BCF0E944F
:103D10009610DF91CF911F910F91FF90EF90DF9060
:103D2000CF90BF90AF909F9008950E942314882356
:103D300021F380E00E94E81D0E944718CC249B2CB0
:103D4000DDCF8EE00E94F713882309F4BACF2FEF5E
:103D5000B21609F4B6CFBA94B4CF88E00E94901698
:103D6000C6CFB394AECF282FF89495E028980000E2
:103D70000000000000009EBD0DB407FEFDCF000056
:103D80000000000000001EBC0DB407FEFDCF8EB584
:103D9000289A000000000000000080FDE7CF28986E
:103DA0000000000086E08EBD0DB407FEFDCF0000D0
:103DB0000000289A00000000000000002898000081
:103DC000000082E08EBD0DB407FEFDCF7EBD0DB4B8
:103DD00007FEFDCF6EBD0DB407FEFDCF2EBD0DB4A9
:103DE00007FEFDCF00000000289A78940895382F30
:103DF000F89425E0289800000000000000002EBD87
:103E00000DB407FEFDCF00000000000000001EBC46
:103E10000DB407FEFDCF8EB5289A0000000000000B
:103E2000000080FDE7CF28980000000083E08EBDF1
:103E30000DB407FEFDCF9EBD0DB407FEFDCF3EBD08
:103E40000DB407FEFDCF000000001EBC0DB407FE40
:103E5000FDCF8EB5289A78940895892F8F7184FDAF
:103E6000806E0895EF92FF920F931F93FA01D9018C
:103E700086958083862F90E08F70907095958795BA
:103E800095958795959587958C93862F8770F801E2
:103E9000808362956F70F70160831F910F91FF908F
:103EA000EF900895FC0130E022953295307F322763
:103EB000207F322720838081660F660F660F640F94
:103EC0006F70862B8083089580917004882349F059
:103ED00087FD0EC083E00E94581684E00E94901671
:103EE000089583E00E94901684E00E949016089541
:103EF00083E00E94901684E00E9458160895962F41
:103F0000803110F08FEF0895682F70E0660F771FF3
:103F10006F5F734F892F0E94B31E80E008959B014D
:103F2000803120F5682F70E0FB01EE0FFF1FEB5290
:103F3000FC4F8081918128173907A0F0009749F044
:103F40008150660F771F6050744F0E94B31E80E04F
:103F5000089580E0660F771F6050744F0E94B31E73
:103F600080E00895C901009759F7F3CF8FEF0895C6
:103F7000803198F470E06050784F90E0002496957E
:103F800087950794969587950794982F802D680FAD
:103F9000791F8CE06030780710F08FEF0895842F40
:103FA0000E94B31E80E00895EF92FF920F931F933B
:103FB000CF93DF93C82FD0E0CC0FDD1FCC0FDD1FD8
:103FC000CC0FDD1FC60FD11DC05CDF4FCC0FDD1F36
:103FD000C295D295D07FDC27C07FDC27EE24FF245A
:103FE0008701000F111F06581A4FF8018081918137
:103FF000892FBE010E94B31EF80180819181219614
:10400000BE010E94B31E0894E11CF11C2196F0E150
:10401000EF16F10429F7DF91CF911F910F91FF90D7
:10402000EF90089590E0880F991F8F5F934F0E9443
:10403000F71E90E008950F931F93082F10E0000FD4
:10404000111FC8018050944F0E94F71E90E0019606
:104050000B521C4FF801208131818217930708F41D
:104060009C01C9011F910F9108958091E9048093EB
:10407000AB058091AB050E941B209093A605809311
:10408000A5058091AB050E9412209093AD05809309
:10409000AC052091AC053091AD058091A5059091BE
:1040A000A6052817390720F01092AD051092AC052F
:1040B00080919A0590919B05E091AB05F0E0EE0FA1
:1040C000FF1FEB52FC4F608171810E9495499093D4
:1040D0009B0580939A050895803198F470E06050B4
:1040E000784F90E00024969587950794969587954C
:1040F0000794982F802D680F791F8CE06030780727
:1041000010F08FEF0895CB010E94F71E0895EF92F3
:10411000FF920F931F93CF93DF93E0909A05F09057
:104120009B050894E11CF11C80E00E943614882352
:10413000C9F400E08091AE05813029F180E00E9451
:104140000D14882329F08091AE05882309F0BFC0A3
:10415000013009F4E7C0DF91CF911F910F91FF90DB
:10416000EF90089581E08093AE051092AA05109219
:10417000A9058093770482E20E94901601E0809165
:10418000AE058130D9F60E945415282F8823B9F046
:1041900021508091A9059091AA057C01EE0CFF1C8D
:1041A000EE0CFF1CEE0CFF1C880F991FE80EF91E89
:1041B000E20EF11CF092AA05E092A90501E087E168
:1041C0000E94F713882341F0E090AC05F090AD0514
:1041D0000894E11CF11C01E083E00E94F71388239E
:1041E00029F0E090A505F090A60501E089E00E9485
:1041F000F713882309F0A2C089E00E940D148823D8
:1042000009F0BAC08AE00E94F713882309F0A5C01C
:104210008AE00E940D14882309F490CF8CE10E945B
:104220009016E091AB052091A5053091A605F0E030
:10423000EE0FFF1FEB52FC4F808191812817390749
:1042400008F07CCF8091A5059091A60501969093EA
:10425000A6058093A5058091AB056091A505709199
:10426000A6050E948F1F8091AB050E941B20909392
:10427000A6058093A5056091A5057091A6056150DE
:10428000704080919A0590919B0586179707D8F406
:10429000EB01219701C0E9018091AB051C2F6C2F28
:1042A0000E946C20482F8091AB051F5F612F0E94F8
:1042B000B81F9E012150304080919A0590919B0536
:1042C0008C179D0740F388E080937A0437CF82E211
:1042D0000E945816109277041092AE0581E08093E8
:1042E0007A042091A9053091AA0521153105A9F07C
:1042F000E091AB05F0E0EE0FFF1FEB52FC4F808129
:1043000091818217930748F02150304030939B05EC
:1043100020939A0587E080937A0410924604013036
:1043200009F019CFC7010E94070200934604DF91EC
:10433000CF911F910F91FF90EF9008958BE10E9414
:1043400058161092AA051092A905E0909A05F090CF
:104350009B050894E11CF11C4FCF8CE10E9458167C
:104360001092AA051092A905E0909A05F0909B057D
:104370000894E11CF11C4CCF8BE10E949016C09177
:104380009A05D0919B0521968091A5059091A6054F
:10439000C817D90708F036CF8091AB051C2F6C2FBA
:1043A0000E946C20482F8091AB051150612F0E9414
:1043B000B81F21968091A5059091A605C817D90729
:1043C00058F38091A5059091A60501979093A605B5
:1043D0008093A5058091AB056091A5057091A60518
:1043E0000E948F1F8091AB050E941B209093A60511
:1043F0008093A50588E080937A0404CFEF92FF9222
:104400000F931F938091E9048093AB058091AB05D6
:104410000E941B209093A6058093A5058091AB0573
:104420000E9412209093AD058093AC052091AC05BD
:104430003091AD058091A5059091A6052817390703
:1044400020F01092AD051092AC0580919A059091E4
:104450009B05E091AB05F0E0EE0FFF1FEB52FC4F28
:10446000608171810E94954990939B0580939A0584
:104470008091AB0560919A0570919B050E946C201C
:104480008093A2058091AB056091A20549EF55E0AC
:1044900021EB35E003EB15E0E5ECEE2EE6E0FE2E39
:1044A0000E94321F81E0809341060E94FC29809186
:1044B000C5068093CC061F910F91FF90EF90089551
:1044C000AF92BF92CF92DF92EF92FF920F931F9322
:1044D000CF93DF93C82EDD24CC0CDD1CCC0CDD1C6F
:1044E000CC0CDD1CC60ED11C80E490E0C80ED91E99
:1044F000CC0CDD1CC294D29410EFD122DC24C1225A
:10450000DC24AA24BB24C6010E94F71ED82FC0E0D9
:104510007501EE0CFF1CEAE7F5E0EE0EFF1EF70159
:10452000D183C08300811181C60101960E94F71ECC
:1045300090E0082B192BF701118300830894A11C2C
:10454000B11C82E090E0C80ED91E90E1A916B1041A
:10455000D1F6DF91CF911F910F91FF90EF90DF90F7
:10456000CF90BF90AF9008951092A40584E20E946E
:1045700090160E9407170E949E1810923F0680E036
:104580000E94E81D08951092A30510923F06109214
:104590009C0580E00E94E81D0E9407170E949E185B
:1045A0000E946E1508958091A0059091A105682F35
:1045B00067709695879596958795969587958F7050
:1045C0000E94CB2D6091A0057091A1059B0140E058
:1045D00050E0DA01C90180709078A070B070892F26
:1045E0009A2FAB2FBB2780938104DA01C901807019
:1045F0009074A070B070892F9A2FAB2FBB27809337
:104600007F042070307240705070232F342F452F5C
:104610005527209380041092B405872F8F7184FD55
:10462000806E089581E08093A30581E20E94581670
:1046300010927F0480917F04809380048091800495
:104640008093810410929C0510923F0680917A0518
:1046500090917B059093A1058093A0058F5F9F4F5C
:1046600089F01092A8051092B40510928D040E9452
:10467000D3228093700480913D0480FDFCCF81E0C3
:1046800080939C050E941C17089581E08093A405E7
:1046900084E20E9458160E941C170895DF92EF9240
:1046A000FF920F931F9380912B07882309F487C2F1
:1046B00084E00E94802A10929F0580919F0580933C
:1046C0009E051092AE051092AA051092A9050E94AF
:1046D000FE218091DD0660911E0740913A062091EF
:1046E000400604E816E00E94072D80913A0660918A
:1046F00040064091B305209141060091B705E09036
:10470000B1050E94561957E0D52E07C0113009F4A3
:10471000FFC00E949E2C8823D9F00E94A6150E94FB
:104720007C0C1091C4061330E9F0143078F3143087
:10473000E9F11D3071F781E00E94B0338091C40629
:104740008D3039F3109285040E949E2C882329F71E
:104750000E946D2C0E94A6150E947C0C1091C4062C
:10476000133019F70E94862A882309F09EC10E94FF
:10477000F82B882321F010927704109285040E9470
:104780008C14882331F2182F11500E944718812F62
:104790000E941E181093C50680912B07882309F0EC
:1047A000B8CF8091C5068093CC06B3CF0E94862AED
:1047B000882309F05CC18091AE05882309F44AC1C1
:1047C0000E94872083E00E943614882309F03BC1B1
:1047D00087E10E943614882309F02EC186E10E94E9
:1047E0003614882309F468C080914106882309F0B3
:1047F000B0C18091C5068093CC06E0909A05F090F8
:104800009B0580919F05882309F090C18091400607
:10481000882309F44AC010E020911E0730913A061F
:104820008091CC0690E082959295907F9827807F2A
:1048300098278093A2058091A205220F220F220FB4
:10484000230F210F2F70282B2093A2058091AB05F9
:1048500060919A0570919B054091A2050E94B81F36
:104860001F5F80919A0590919B05019690939B05FF
:1048700080939A050894E11CF11C80919A0590910F
:104880009B05E091AB05F0E0EE0FFF1FEB52FC4FF4
:10489000608171810E94954990939B0580939A0550
:1048A00080914006181708F4B7CF80919E058823A1
:1048B00009F052C1D0927A0480917A04873009F4C9
:1048C00007C180917A04883009F459C180917A0433
:1048D000813009F4AEC08091C406843011F010928A
:1048E000850480912B07882309F4DBC08091840420
:1048F000813009F00ECF109284040E94CB298823C6
:1049000009F407CF1F910F91FF90EF90DF9008956A
:104910000E94862A882309F073C00E94872083E0C2
:104920000E943614882339F583E00E940D148823F1
:10493000F1F49091AB058091E904981711F00E9471
:10494000FE218091C406813011F01092850480917F
:104950002B07882309F0B8C00E94CB29882309F4CB
:10496000D8CE1F910F91FF90EF90DF90089583E2D2
:104970000E949016DECF10929B0510929A058091AE
:10498000AB0560919A0570919B050E946C20809305
:10499000A2058091AB056091A20549EF55E021EB9E
:1049A00035E003EB15E0A5ECEA2EA6E0FA2E0E9416
:1049B000321F81E0809341068091C5068093CC062A
:1049C0000E94FC298091DD0660911E0740913A0605
:1049D0002091400604E816E00E94072D80913A06D7
:1049E000609140064091B305209141060091B705C2
:1049F000E090B1050E94561983E20E94581694CFA8
:104A00000E94071782E20E9458161093850481E2E3
:104A10000E94901680913A06609140064091B3053D
:104A20002091410600913A06E090B1050E94561986
:104A300074CF10927A044FCF81E080939F0580E07D
:104A40000E947416CBCE81E080939E0583E20E9483
:104A50007416BECE0E948B2C9091AB0596959093C8
:104A6000F304882309F0ACCE0E94B033A9CE0E9493
:104A7000071782E20E94581681E08093850481E244
:104A80000E94581680913A06609140064091B30505
:104A90002091410600913A06E090B1050E94561916
:104AA0008ACE81E00E94802A21CF0E94071711E060
:104AB0001093770484E20E9458168091C5060E94E4
:104AC0001E181093850453CE84E00E94802A44CFA0
:104AD0008091AB0560919A0570919B050E946C20B6
:104AE0008093A2058091AB056091A20549EF55E046
:104AF00021EB35E003EB15E095ECE92E96E0F92E7D
:104B00000E94321F11E01093410680913A06609195
:104B100040064091B305209141060091B705E09011
:104B2000B1050E94561910937A04D0CE10929F05B9
:104B30008091AB056E2D0E947F1F8091AB050E9476
:104B400012209093AD058093AC0580E00E949016F2
:104B50005DCE0E94FC294DCE10929E058091AB0542
:104B6000B7010E948F1F8091AB050E941B2090937C
:104B7000A6058093A50583E20E9490169BCE8091A6
:104B8000AB0560919A0570919B050E946C20809303
:104B9000A2058091AB056091A20549EF55E021EB9C
:104BA00035E003EB15E0B5ECEB2EB6E0FB2E0E94F2
:104BB000321F81E08093410610927A0487CE81E013
:104BC0000E94802A78CDEF92FF920F931F938091DD
:104BD0002B07882309F4ACC184E00E94802A10923C
:104BE0009F0580919F0580939E051092AE051092BF
:104BF000AA051092A9050E94FE218091DD06609110
:104C00001E0740913A062091400604E816E00E94F3
:104C1000072D80913A06609140064091B30520919E
:104C200041060091B705E090B1050E94561908C0F1
:104C3000143009F461C00E949E2C882309F492C0AC
:104C40000E94A6150E947C0C1091C406113081F7B9
:104C50000E94862A882309F0DAC083E00E94361475
:104C6000882309F0F5C083E00E940D14882309F021
:104C700039C180E00E943614882309F03CC180E0ED
:104C80000E940D14882309F04BC19091AB058091CF
:104C9000E9049817E1F00E94FE218091DD06609101
:104CA0001E0740913A062091400604E816E00E9453
:104CB000072D80913A06609140064091B3052091FE
:104CC00041060091B705E090B1050E945619809108
:104CD000C406813011F01092850480912B0788233F
:104CE00009F043C00E94CB29882309F4A4CF1F9167
:104CF0000F91FF90EF9008950E94862A882309F073
:104D000065C086E10E943614882309F053C083E011
:104D10000E943614882309F041C080E00E943614B6
:104D2000882339F580E00E940D14882379F580915D
:104D3000C406843011F01092850480912B078823DB
:104D400009F461C080918404813009F074CF10921D
:104D500084040E94CB29882351F60E949E2C88232C
:104D600009F06ECF0E946D2C6BCF84E00E94802AE8
:104D7000B9CF11E01093AE0582E20E949016109315
:104D8000460480E00E940D14882389F282E20E948A
:104D900058161092AE0510924604C9CF81E0809358
:104DA0009E0583E20E94581610929F0580E00E94A3
:104DB0009016B3CF81E080939F0580E00E94581643
:104DC00010929E0583E20E949016A1CF0E940717C1
:104DD00082E20E94581681E08093850481E20E945D
:104DE000581680913A06609140064091B305209193
:104DF000410600913A06E090B1050E94561981E003
:104E00000E9443027ECF81E00E94802A9BCF0E94B5
:104E1000071782E20E9458161093850481E20E94CF
:104E2000901680913A06609140064091B30520911A
:104E3000410600913A06E090B1050E94561981E0C2
:104E40000E94430283E00E943614882309F40BCFAA
:104E500010929B0510929A058091AB0560919A057E
:104E600070919B050E946C208093A2058091AB05F8
:104E70006091A20549EF55E021EB35E003EB15E029
:104E800075ECE72E76E0F72E0E94321F81E08093CA
:104E900041068091C5068093CC060E94FC29809132
:104EA000DD0660911E0740913A062091400604E815
:104EB00016E00E94072D80913A06609140064091CD
:104EC000B305209141060091B705E090B1050E941D
:104ED000561983E20E94581683E00E940D1488231D
:104EE00009F4C7CE83E20E94901680E00E94361437
:104EF000882309F4C4CE11E01093AE0582E20E942B
:104F0000901680919A0590919B0501960E94070248
:104F10001093460480E00E940D14882309F4B5CE56
:104F200082E20E9458161092AE0510924604ADCE51
:104F300081E00E94802A53CEEF920F931F9310922C
:104F4000720480912B07882309F421C284E00E9417
:104F5000802A10929F0580919F0580939E05109254
:104F6000AE051092AA051092A9050E94352007C02F
:104F7000113009F493C00E949E2C8823D9F00E941E
:104F8000A6150E947C0C1091C4061330E9F0143071
:104F900078F31430E9F11D3071F781E00E94B033ED
:104FA0008091C4068D3039F3109285040E949E2CA6
:104FB000882329F70E946D2C0E94A6150E947C0C64
:104FC0001091C406133019F70E94862A882309F02D
:104FD000B0C00E94F82B882321F010927704109221
:104FE00085040E948C14882331F2182F11500E94DE
:104FF0004718812F0E941E181093C50680912B0719
:10500000882309F0B8CF8091C5068093CC06B3CF32
:105010000E94862A882309F0D5C08091AE05882396
:1050200009F4C3C083E00E943614882329F08091DC
:105030007204813009F487C187E10E943614882305
:1050400009F08CC080E00E943614882309F092C0D9
:1050500080E00E940D14882309F09AC08091C40654
:10506000843011F01092850480912B07882309F475
:105070006FC080918404813009F07DCF1092840448
:1050800080917204882309F076CF0E94CB2988236F
:1050900009F471CF1F910F91EF9008950E94862A15
:1050A000882309F0D9C08091AE05882309F4F9C09E
:1050B00083E00E943614882379F081E080937204A3
:1050C00080917204882309F432C183E20E94581649
:1050D00010929B0510929A0580E00E943614882356
:1050E00009F0ECC01091AE05113009F4FFC080E06A
:1050F0000E940D14882309F089C09091AB0580911E
:10510000E904981711F00E9435208091C40681307F
:1051100011F01092850480912B07882309F4B5CFF4
:1051200084E00E94802A0E94CB29882309F423CF9F
:10513000B1CF0E94071711E01093770484E20E9418
:1051400058168091C5060E941E181093850441CF01
:1051500081E00E94802A109272048BCF81E08093BC
:105160009F0580E00E94741680E00E943614882318
:1051700009F46ECF11E01093AE0582E20E94901602
:105180001093460480E00E940D14882309F466CF32
:1051900082E20E9458161092AE058091460481303A
:1051A00009F4E6C01092460459CF0E948B2C9091CE
:1051B000AB0596959093F304882309F033CF0E94B2
:1051C000B03330CF0E94071782E20E94581681E068
:1051D0008093850481E20E94581680913A0660917E
:1051E00040064091B3052091410600913A06E090B7
:1051F000B1050E94561980917204882309F49BC05E
:1052000083E20E9474160E94671807CF82E20E9410
:1052100058161092AE052091A9053091AA052115C6
:10522000310591F0E091AB05F0E0EE0FFF1FEB527E
:10523000FC4F808191818217930730F021503040DC
:1052400030939B0520939A0580914604813009F4A0
:1052500080C01092460451CF0E94071782E20E943C
:1052600058161093850481E20E94901680913A06A8
:10527000609140064091B3052091410600913A06A5
:10528000E090B1050E94561980917204882309F4B8
:1052900056C083E20E9458168091AE05882309F01B
:1052A00007CF0E948B2C9091AB0596959093F304B9
:1052B000882309F0FDCE0E94B033FACE11E010939E
:1052C000AE051092AA051092A90582E20E949016DE
:1052D00080919A0590919B0501960E940702109378
:1052E00046041091AE05113009F001CF0E9454150B
:1052F000482F882309F4FBCE41502091A905309115
:10530000AA05C901880F991F880F991F880F991F37
:10531000220F331F820F931F840F911D9093AA05B4
:105320008093A9050E94070210934604E0CE83E211
:105330000E949016CDCE83E20E94901664CF83E245
:105340000E949016B0CE80939E0583E20E9458166C
:1053500073CE80913A06609140064091B30520914A
:10536000410600913A06E090B1050E94561971CFAE
:1053700080913A06609140064091B3052091410624
:1053800000913A06E090B1050E9456190BCF81E0DA
:105390000E94802ADECD9091E8048091EE04891766
:1053A00031F08091E8048093EE0481E0089580E07C
:1053B000089580914106882391F08091F9058093AA
:1053C000DD068091B10580931E078091B30580931F
:1053D0003A068091410680934006109241068091E2
:1053E0004006882329F08091400680934006089566
:1053F00081E08093400608958091F9058093DD0651
:105400008091B10580931E078091B30580933A0681
:1054100080914106809340061092410608958330A2
:1054200059F0843050F0843029F08091C506809383
:10543000CC0608951092C50608958230B0F70895FD
:10544000FC0187858F708D30C1F030E020E190E065
:1054500080818F708E3061F09F5F31969217C0F31C
:10546000892F913118F48150832B089580E1FBCF6F
:105470009923B1F780E0832B089530E12FE0E7CF47
:105480001F93DF93CF930F92CDB7DEB7162F0E94F5
:10549000202A898389818F708F5F8093F70310930F
:1054A000B705898184FD08C08CE08093F5030F90D7
:1054B000CF91DF911F91089580E18093F5030F90C4
:1054C000CF91DF911F910895E82FF0E0EF73F07016
:1054D000E750FC4F808108954093B5056093F8052F
:1054E0008093C40681E080933D060895882339F0B7
:1054F0008091F8058093C40681E080933D0608956D
:105500008093C40681E080933D06089580913D0616
:10551000882319F010923D0681E008953F924F9242
:105520005F926F927F928F929F92AF92BF92CF9233
:10553000DF92EF92FF920F931F93CF93DF93462E4C
:105540004A015901662309F4C4C09C01E9011FEF17
:10555000DD2400E0FF2466247724B2E05B2E3324B0
:105560003394CE010E94202AF301E853F94F80833F
:10557000C0802FE0C222C39440E050E012C01E253C
:105580001F7BF1F4F501E00FF11D3082FF2009F0DF
:1055900070C0DD24D3940F5F4F5F5F4F1E2D4C15FD
:1055A00088F5642FFE01E40FF51FE0802E2D30E01A
:1055B000C9018F7090700F9709F455C0DD20F9F67E
:1055C000F501E00FF11D5082EF2DF0E0D401AE0F98
:1055D000BF1FEC926295607FEE5BF94F6083F3949E
:1055E0000024220F331F001C220F331F001C232F07
:1055F000302DDD24D394D2220F5F4F5F5F4F1E2DDD
:105600004C1578F20894611C711C6096641408F4BF
:10561000A8CF003408F061C08F2DF501E00FF11D17
:1056200010820F5F0034C8F39FE39F1550F09FEF87
:10563000EF2DF0E0EE5BF94F9083F3942FE32F15FD
:10564000B8F7DF91CF911F910F91FF90EF90DF900E
:10565000CF90BF90AF909F908F907F906F905F9012
:105660004F903F900895F501E00FF11D1082DD2469
:1056700092CFEF2DF0E03197E80DF91DE082FA941A
:10568000EF2DF0E0F394EE5BF94FA081AF70BA2FED
:10569000BF5F808182958F70682F70E0CB018B0F88
:1056A000911D40970CF0BA2F0024220F331F001CCD
:1056B000220F331F001C232F302DDD24D394D22240
:1056C00062957295707F7627607F7627B62BB083C0
:1056D00062CF00E0FF2480E0A0CF8F2DA5CF2F92D6
:1056E0003F924F925F926F927F928F929F92AF9272
:1056F000BF92CF92DF92EF92FF920F931F93CF93BF
:10570000DF935C01562E3A016901662309F45DC0FE
:10571000482EEC0130E060E0EE24FF24FA9480E0B3
:1057200000E010E05FE04EE0342E2DE0222E98ECF9
:10573000892E96E0992E800E911EF40170817F7063
:105740007F5FDE0190E0442D41950BC05C932230D9
:1057500089F0E42EEA0E3F5F9F5F1196822F971724
:10576000D0F4F601E30FF11D2081213079F7882371
:1057700049F45C93F301E60FF11DF0806F5FFC923A
:1057800022E0E7CF5C93F501EE0DF11D808180648E
:105790008083FC92DECF903158F4FE01E90FF11DB9
:1057A00030829F5F05C0FE01E90FF11D50839F5FAE
:1057B0009031C8F3F401808184FD2F860F5F1F4F65
:1057C0006096822F051508F4B2CFDF91CF911F911B
:1057D0000F91FF90EF90DF90CF90BF90AF909F9090
:1057E0008F907F906F905F904F903F902F90089593
:1057F0008091B5050E940D14882339F08091F80539
:105800008093C40681E080933D0608951092A4051C
:1058100084E20E9490161092740480E00E94901618
:105820000E949E180E94A2170E941C178091F204E9
:105830000E942A1780E00E94E81D089581E080936D
:10584000A40584E20E9458160E941C1780E00E9462
:105850002A1780E00E94E81D089510923F060E94DA
:10586000A2170E941C170E949E188091F2040E94A9
:105870002A1710923B0681E20E94901680E00E9457
:10588000E81D10922B078CEF0E944710089510928C
:10589000B40581E080933B0681E20E94581680E0C7
:1058A0000E94E81D80913C04882321F480913D04EE
:1058B00080FDFCCF10923D04109258041092990480
:1058C0008091990480939B0481E080933F068093AC
:1058D0002B078AEF0E944710089580918504882342
:1058E00011F480E0089581E00E943614882321F0AD
:1058F00081E080938604089581E00E94F713882355
:1059000081F380E00E94E113882359F382E08093C1
:10591000860481E0089588E00E94E113882369F0FD
:105920009091C40688E08093B5059093F80583E0D4
:105930008093C40681E080933D06089580913C04E5
:10594000823011F080E008950E9476108093200745
:1059500080E00895AF92BF92CF92DF92EF92FF92D4
:105960000F931F93CF93DF935B01C82EDD24C29466
:10597000D29450EFD522DC24C522DC24EE24C0E0F2
:10598000D0E0FF24F39405C02196F394F1E1FF16D3
:10599000B1F085010C0F1D1FC6018C0F9D1F0E94C9
:1059A000F71EF8018083EE2079F780818F708E30AA
:1059B00059F7EF2C2196F394F1E1FF1651F7EE2001
:1059C000A1F490E1F50187858F708D30B9F0892FB2
:1059D00081508F70DF91CF911F910F91FF90EF90C9
:1059E000DF90CF90BF90AF9008959E2D915051F7CA
:1059F00091E0F50187858F708D3049F7903110F077
:105A00008EE1E8CF892F81508F708061E3CFBF9204
:105A1000CF92DF92EF92FF920F931F93CF93DF937A
:105A20006801E82EFF24EE0CFF1CE60EF11CEE0CC4
:105A3000FF1CEE0CFF1CEE0CFF1CE40EF11CE294AC
:105A4000F29470EFF722FE24E722FE2430E0229544
:105A50003295307F3227207F3227B22E222379F0F1
:105A6000C0E0D0E086010C0F1D1FC7018C0F9D1FE9
:105A70000E94F71EF80180832196CB1598F3DF91E1
:105A8000CF911F910F91FF90EF90DF90CF90BF903B
:105A90000895EF92FF920F931F93CF93DF93182FE8
:105AA000062F0E946718E12EFF24EE0CFF1CEE0C5F
:105AB000FF1CEE0CFF1CE00EF11CE294F294A0EF30
:105AC000FA22FE24EA22FE24C0E0D0E0FE01E353E5
:105AD000F94F8081BE016E0D7F1D0E94B31E21967D
:105AE000C031D10599F70E946718DF91CF911F91BE
:105AF0000F91FF90EF900895CF92DF92EF92FF9277
:105B00000F931F93CF93DF93E22E6801082F10E0CD
:105B1000000F111F060F111D000F111F000F111F85
:105B2000000F111F040F111D02951295107F1027F1
:105B3000007F1027FF24E294F29480EFF822FE24E5
:105B4000E822FE24FE2C82E00E9458160E9467186C
:105B5000EE2099F0C0E0D0E0F601EC0FFD1F80814F
:105B6000B8016C0F7D1F0E94B31E82E00E943C0FA3
:105B70000E947C0C2196CF1578F382E00E9490164B
:105B80000E946718DF91CF911F910F91FF90EF90C6
:105B9000DF90CF900895EF92FF920F931F93CF93D2
:105BA000DF93182F062F0E946718E12EFF24EE0CBA
:105BB000FF1CEE0CFF1CEE0CFF1CE00EF11CE2942F
:105BC000F29440EFF422FE24E422FE24C0E0D0E070
:105BD000CE018E0D9F1D0E94F71EFE01E353F94F6B
:105BE00080832196C031D10599F71092740480E02A
:105BF0000E94AD160E946718DF91CF911F910F91FF
:105C0000FF90EF90089580913C04882349F40E940E
:105C1000A90080913C04813049F00E948C130895C2
:105C20000E94AA0080913C048130B9F70E9493132E
:105C300008950F931F938091C5068093CC068091A1
:105C400041068823C9F08091F9058093DD06809193
:105C5000B10580931E078091B30580933A06809129
:105C6000410680934006109241068091770482306D
:105C700088F01F910F91089590911E078091B105B2
:105C80009817B9F380917704823098F78091B10525
:105C900080931E078091DD0660911E0740913A06B1
:105CA0002091400604E816E00E94072D60913A0614
:105CB0008091C6069091C7060E94402A1F910F91BD
:105CC000089510922B0780E00E94E81D8CEF0E943F
:105CD000471080913C04813011F00E9462131092B1
:105CE0008206109299048091990480939B041092EB
:105CF000B20584E896E09093C7068093C60680912B
:105D0000EE048D3031F0833021F08B3011F087308C
:105D100011F40E94192E80914A04882361F4809125
:105D20004904882309F40895809149040E942110B0
:105D300010924904089580914A040E942110109203
:105D40004A04EDCF4F925F926F927F928F929F9213
:105D5000AF92BF92CF92DF92EF92FF920F931F9379
:105D6000CF93DF9381E08093C40680933D0610E0DB
:105D7000C0E0D0E0BB24FF24F394AA24AA9442E01C
:105D8000E42E34E0932E23E0822E90E2792E80E1FF
:105D9000682E0FE0502EB1E14B2E0E94A6150E94F6
:105DA0007C0C8091C406873009F4DFC0883008F08D
:105DB0007EC0843009F46FC2863009F42EC281306F
:105DC00061F780913D06882331F010923D060E94D4
:105DD00007170E94671887E10E943614882361F034
:105DE0008091C40697E19093B5058093F80587E00C
:105DF0008093C406F0923D0688E00E943614882302
:105E000061F08091C40698E09093B5058093F80501
:105E100086E08093C406F0923D0681E00E9436142D
:105E2000882351F08091C406F092B5058093F8055F
:105E30009092C406F0923D068EE00E9436148823AC
:105E400059F09091C4068EE08093B5059093F805C3
:105E50005092C406F0923D0682E00E9436148823D8
:105E600051F08091C406E092B5058093F8056092E8
:105E7000C406F0923D069091E8048091EE048917E3
:105E800009F48BCF8091E8048093EE04DF91CF91E9
:105E90001F910F91FF90EF90DF90CF90BF90AF9048
:105EA0009F908F907F906F905F904F90089580317A
:105EB00009F42FC1813109F4BEC08F3009F06DCFD4
:105EC00080913D06882349F010923D06F0927A04B5
:105ED0008091E9048093790410E08091B5050E94D7
:105EE0000D14882349F08091F8058093C406F09240
:105EF0003D06112309F0DBC20E94DA14882369F001
:105F0000982F9150933048F48091AD04981729F060
:105F10009093AD04F0927A0411E08091AD04813049
:105F200009F48BC280917A04882309F436CF109249
:105F30007A040E9410180E941C178091AD048F5F94
:105F40000E94B0178091AD04813009F026CF809176
:105F5000B00481500E942A170E94A6150E947C0C52
:105F60008091C406873009F021CF80913D068823B7
:105F700039F010923D06F0927A0480E00E945816A3
:105F80008091B5050E940D14882351F08091F80589
:105F90008093C406F0923D0680917A0481FDD0C2C0
:105FA0000E94DA14882389F0982F9150933068F476
:105FB00080913C04981749F090933C040E94032E72
:105FC00080917A04836080937A0483E00E94F713BF
:105FD000882379F080917D048F5F80937D04809188
:105FE0007D04817080937D0480917A048360809326
:105FF0007A0486E10E94F713882309F0AEC18091EC
:106000007A0480FFCACE80917A048E7F80937A04CE
:106010000E94101880913C048F5F0E94B01783E2A9
:106020000E94901680917D04882309F06FC083E25E
:106030000E9458166BC080913D068823C9F01092CB
:106040003D06F0927A04A09278048091A3048130F6
:1060500009F43FC2823009F427C2843009F421C216
:10606000883011F48092780482E00E94581610E083
:106070008091B5050E940D14882349F08091F805A0
:106080008093C406F0923D06112309F025C20E94B8
:10609000DA14882341F1982F9150943020F58091A3
:1060A0007804981701F190937804F0927A04809123
:1060B0007804882309F06AC241E080917804823034
:1060C00009F46AC280917804833009F46BC2242FEA
:1060D00030E0C901880F991F820F931F880F8093AA
:1060E000AA044093A30480917A04882309F455CE2E
:1060F00010927A040E94101880917804843008F07D
:1061000005C2809178048F5F0E94B0170E946718C3
:1061100044CE80913D06882359F010923D06F092BE
:106120007A041092F803F092780410E0C0E0D0E016
:106130008091B5050E940D148823B1F08091F80577
:106140008093C406F0923D06112351F080917804AB
:10615000813009F45DC280917804823009F425C24F
:1061600010924604F092F80380E00E94F71388230F
:1061700061F080917804823041F0E092780482E20C
:106180000E947416F0927A0410E00E945415282F91
:10619000882389F0CE01880F991F880F991F880FD7
:1061A000991FCC0FDD1FC80FD91F2150C20FD11D61
:1061B000E0927A0411E000917804023009F459C1A8
:1061C00080917A04882309F4E8CD809178048130A5
:1061D00009F48CC180917804823009F0DECD809181
:1061E0007A04823009F042C20C2F8BE10E94901693
:1061F0008CE10E949016002339F0B7FC62C21B1498
:106200001CF48CE10E945816802F90E00E94070237
:10621000F092460410927A04C0CD80913D06882306
:1062200039F010923D0610927A041092780410E032
:106230008091B5050E940D14882349F08091F805DE
:106240008093C406F0923D06112309F06CC1809141
:106250007804882309F4D9C020917804213009F406
:10626000B7C020917804223009F486C080917A0466
:10627000813009F4A2C080917A04823009F08DCD7A
:1062800010927A040E941C178091B3040E942A176E
:106290000E94671882CD80913D06882339F01092C4
:1062A0003D06F0927A041092780410E08091B505D2
:1062B0000E940D14882331F18091F8058093C40663
:1062C000F0923D061123E1F080917804882311F4C7
:1062D000F092780480917804813210F07092780402
:1062E0009091000280917804981751F08091780481
:1062F000809300026091000287E090E00E946C02AF
:10630000109246040E945415382F882389F08091FA
:1063100078042AE0829FC001112480937804809140
:1063200078048150830F80937804E0927A0411E01E
:1063300080917A04882309F430CD909100028091F5
:106340007A04823009F413C1892F90E00E94070279
:10635000F092460410927A0420CD9091F80587E1DE
:106360008093B5059093F8054092C406F0923D06DF
:1063700080E00E94901643CE9091E90480917904C8
:10638000981759F08091E9048093790420937A0456
:10639000809179048093B30411E089E00E940D1488
:1063A000882309F463CF109278048BE10E94901641
:1063B00080917A04813009F05ECF10927A040E94B5
:1063C0001C178091C6040E942A170E946718E5CC0A
:1063D0009091E90480917904981759F08091E9042B
:1063E0008093790420937A04809179048093C60481
:1063F00011E08AE00E940D14882309F432CF109234
:1064000078048CE10E9490162CCF8AE00E94F7134A
:10641000882309F0AFC089E00E94F713882309F4AC
:106420001BCF8BE10E945816E0927804E0927A0428
:106430008091E904809379040FCF90917904809141
:10644000E904981709F46ECD8091E90480937904EA
:10645000909179049F5F923008F418C18091B00444
:10646000981709F45FCD9093B004F0927A0411E08C
:1064700059CD89E00E94F713882331F01B1424F4CE
:1064800000937A04BB24BA948AE00E94F71388230D
:1064900009F496CEB7FE94CEE0927A04BB24B3946E
:1064A0008FCEE0927804E0CDF0927804DDCD80913B
:1064B000B0046091AD0490E0019782959295907F31
:1064C0009827807F9827682B8AE090E00E946C02D2
:1064D00013CD10927804C8CD8EE090E06091A304B3
:1064E0000E946C0282E00E949016D1CD80917A04C5
:1064F000823009F4CDC080918F04909190040E9465
:106500000702F092460410927A0464CE85E00E945D
:10651000B01786E00E94B01787E00E94B01788E0AD
:106520000E94B017F3CD83E090E06091C6040E9412
:106530006C0284E090E06091B3040E946C0287CE0C
:1065400080917D0490E08170907082959295907F0B
:106550009827807F982760913C046F70682B82E0B9
:1065600090E00E946C0280E00E94901619CD9091FC
:106570007804EACE8CE10E945816F0927804F092EA
:106580007A048091E9048093790445CF42E08091B8
:106590007804823009F096CD44E08091780483300D
:1065A00009F095CD48E080E39ACDB7FC81C081E049
:1065B000C536D10508F073C0992787FD90958C9F4B
:1065C00060018D9FD00C9C9FD00C1124BC2C6C2D95
:1065D000772767FD7095872F972F22EE34E040E0F4
:1065E00050E00E946A4960537D4E8C4E9F4F0C2DA7
:1065F000F8946093090270930A0280930B029093BF
:106600000C028DE090E0602F0E946C027894A8CD7F
:10661000C431D10508F440C081E0CD32D80710F074
:10662000CCE2D1E0F89480918F04909190048C1783
:106630009D07D1F0D0939004C0938F0480918F0474
:10664000909190040E94D20280918F0490919004C6
:106650009093A9048093A80460918F047091900492
:1066600085E090E00E947602789475CD8DE090E010
:106670000E946502282F992787FD909597FD1DC0E0
:10668000082F27FD17C0BB24B394AFCD92E0E6CE10
:10669000CE010E94070235CFC4E1D0E0C3CFC0E0F5
:1066A000D0E0BB2460ED72E183E190E000E0A0CF98
:1066B0008FEF7ECFBB24BA9498CD909581959F4F54
:1066C000DFCF8BE10E9458169ACD1F93DF93CF93B3
:1066D0000F92CDB7DEB780E00E94E81D10928206CF
:1066E00010923D041092580410928704109299045D
:1066F0008091990480939B041092B20584E896E0FF
:106700009093C7068093C60610913A060E94202AED
:10671000898389818F708F5F8093F7031093B7050A
:10672000898184FD1BC08CE08093F50383E0809316
:106730002B078AEF0E94471080913C04813011F0B2
:106740000E949A1383E080934404109249041092AB
:106750004A040F90CF91DF911F91089580E1E4CF1B
:10676000EF920F931F93982F882309F495C08130DF
:1067700029F080E01F910F91EF90089580913D06E0
:10678000882309F0F9C00E94DA14882399F1982F20
:10679000915080914106882341F480913A0680937C
:1067A000B3058091DD068093F9058091B3058917C3
:1067B00070F48091B305981B9F5F90934106809180
:1067C0004106853008F446C184E0809341068091FB
:1067D0002B07882309F441C180913A066091400655
:1067E0004091B305209141060091B705E090B105B5
:1067F0000E94561984E10E94F713882309F0DEC035
:1068000085E10E94F713882309F0CEC080912B0701
:10681000882321F590911E078091B1059817F1F01A
:106820008091B10580931E078091DD0660911E075F
:1068300040913A062091400604E816E00E94072D98
:1068400080913A06609140064091B305209141063F
:106850000091B705E090B1050E94561980912B0771
:10686000882329F480914106882309F0D4C00E942E
:10687000F414982F882309F47CCF809178049150E8
:10688000981709F076CF8091F8058093C40681E0CF
:1068900080933D0680E06ECF0E94DA14982F882303
:1068A000D1F584E10E94F713882309F49FC0109268
:1068B000B10588E00E94581681E00E9490168091F0
:1068C0002B07882309F055CF90911E078091B105C1
:1068D000981709F44ECF8091B10580931E078091DF
:1068E000DD0660911E0740913A062091400604E8BB
:1068F00016E00E94072D80913A0660914006409173
:10690000B305209141060091B705E090B1050E94C2
:10691000561980E02FCF8091F3048093F90501E0B0
:1069200000934106192F11501093B30584E10E9482
:10693000E113882309F44BC01092B10588E00E944E
:10694000581681E00E949016109378048091C40636
:106950008093F8058DE08093C40681E080933D0626
:106960001092C50680912B07882309F44FC081E05F
:106970001F910F91EF90089510923D06909385041A
:1069800080913A06609140064091B30520914106FE
:106990000091B705E090B1050E9456190E94DA14E3
:1069A000882309F427CFF3CE81E08093B10588E0F6
:1069B0000E94901681E00E94581628CF1092B105CF
:1069C00088E00E94581681E00E94901619CF85E158
:1069D0000E94E113882309F4B7CF0093B10588E042
:1069E0000E94901681E00E945816AECF85E10E9469
:1069F000F713882309F463CF81E08093B10588E021
:106A00000E94901681E00E94581659CF82E00E94A1
:106A10000F2A81E0ADCF8091F9058093DD0680914A
:106A2000B10580931E078091B30580933A0680914B
:106A3000410680934006109241068091DD066091E8
:106A40001E0740913A062091400604E816E00E9495
:106A5000072D0DCF80914106B8CE8091F905809326
:106A6000DD068091B10580931E078091B305809368
:106A70003A0680914106809340061092410680912B
:106A8000DD0660911E0740913A062091400604E819
:106A900016E00E94072DA0CE2F923F924F925F9258
:106AA0006F927F928F929F92AF92BF92CF92DF921E
:106AB000EF92FF920F931F93DF93CF930F92CDB777
:106AC000DEB70E94A6151092C5068091C506809378
:106AD000CC0680912B07882311F40C94043F84E0AA
:106AE0008093C40681E080933D066624992488241F
:106AF0005524772473945CE0452E43E0342E34E033
:106B0000232E0E94A6150E947C0C1091C4061830FA
:106B1000E9F0193008F04EC0153009F49EC4163063
:106B200008F096C0113009F42FC2143009F40CC4D7
:106B30000E949E2C882329F70E946D2C0E94A61586
:106B40000E947C0C1091C406183019F780913D0604
:106B5000882349F010923D060E94071783E20E94A5
:106B60005816709277048091B5050E940D14882301
:106B7000A1F08091F8058093C40670923D061092B2
:106B800077048091DD0660911E0740913A062091BE
:106B9000400604E816E00E94072D0E94DA148823BC
:106BA00009F00CC50E94F414882311F281500E9450
:106BB0004E19BECF1B3009F4DAC21C30C0F51930B3
:106BC00009F481C21A3009F0B3CF80913D068823C1
:106BD000F1F010923D0680E00E9458160E9467185E
:106BE0008091DD0660911E0740913A062091400693
:106BF00004E816E00E947C2D80E00E9490160E941E
:106C000067182092C40670923D0610927704809116
:106C10007A04882331F02092C40670923D061092C7
:106C20007A0480917A048F5F80937A0481CF1C303C
:106C300009F47AC11D3009F07BCF81E00E94B033A6
:106C40008091C4068D3009F473CF1092850470CF03
:106C5000163009F4F9C0173009F06ACF80913D066B
:106C6000882389F110923D060E9407176091400623
:106C700084E896E04EED56E028EB35E00E948E2A3F
:106C800080E00E94581610927A0489E0809378047C
:106C90001092790480914006882391F020E0E22F41
:106CA000F0E0E853F94F9081809179048F5F9F70F5
:106CB000890F809379042F5F80914006281778F31D
:106CC00066249924552480E00E943614882311F00C
:106CD0006624639488E00E943614882311F082E0D1
:106CE000682E87E10E943614882311F003E0602E9D
:106CF00080917804893009F407C780917804813045
:106D000009F4DBC680917804882309F492C5809148
:106D10007804882329F080917804807F09F45CC08E
:106D2000109178048EE00E94F713882351F080912F
:106D30007804806180937804F5E0F0937A04B2E0FF
:106D40005B2E8FE00E94F713882351F08091780426
:106D500080628093780485E080937A04552453946C
:106D600084E10E94F713882349F0809178048064BD
:106D70008093780495E090937A0455248EE00E94E5
:106D80000D14882339F080917804807E80937804F4
:106D900020927A048FE00E940D14882339F08091AC
:106DA0007804807D8093780420927A0484E10E94A4
:106DB0000D14882339F080917804807B80937804C7
:106DC00020927A0480917A04853009F452C580912A
:106DD0007A04843009F464C580917804883009F419
:106DE00040C480917A0490E083709070892B09F000
:106DF00050C4662009F49CCE6091400684E896E079
:106E00004EED56E028EB35E00E946F2B8091DD06B9
:106E100060911E0740913A062091400604E816E072
:106E20000E947C2D81E0681609F44AC592E069163B
:106E300009F474C0F3E06F1609F07ACE87E080930E
:106E4000C40670923D0674CE80913D068823D9F029
:106E500010923D060E9407176091400684E896E074
:106E60004EED56E028EB35E00E948E2A84E20E9427
:106E7000581610927A0410927904F3E6F09378048D
:106E800066249924882480E00E943614882311F017
:106E90006624639488E00E943614882311F022E06F
:106EA000622E80917804833609F422C5809178049B
:106EB000813009F42CC580917804833009F48AC5A7
:106EC00080917804882309F455C480917A0490E075
:106ED00083709070892B09F01DC4662009F428CEB8
:106EE0006091400684E896E04EED56E028EB35E0F0
:106EF0000E946F2B8091DD0660911E0740913A063B
:106F00002091400604E816E00E947C2D81E068167E
:106F100009F4D6C492E0691609F00ACEE6E0E093DF
:106F2000C40670923D0604CE80913D06882389F008
:106F300010923D069091750480914006981709F4CF
:106F400050C670927A048091F8058093C4067092BE
:106F50003D068091B5050E940D14882309F4E8CD03
:106F60008091F8058093C40670923D0680917A0462
:106F7000882309F4D9C58DE00E94901682E00E9412
:106F800090160E946718D4CD80913D068823E9F0C1
:106F900010923D0680E00E9443020E94071782E2A1
:106FA0000E9458161093850481E20E9490168091E9
:106FB0003A06609140064091B30520914106009148
:106FC0003A06E090B1050E94561980E00E94B03365
:106FD00080E00E94F713882329F085E08093C4069F
:106FE00070923D0683E00E94F713882359F0809148
:106FF000C4063092B5058093F80588E08093C406F6
:1070000070923D0688E00E943614882329F096E0AD
:107010009093C40670923D0687E10E94361488233F
:1070200029F0E7E0E093C40670923D068BE00E94F1
:107030003614882359F09091C4068BE08093B505EF
:107040009093F8058093C40670923D068DE00E94EF
:107050003614882359F09091C4068DE08093B505CD
:107060009093F8054092C40670923D068091C40644
:10707000813011F01092850480912B07882321F034
:107080002092C40670923D069091E8048091EE042F
:10709000891709F44DCD8091E8048093EE040F9098
:1070A000CF91DF911F910F91FF90EF90DF90CF90E4
:1070B000BF90AF909F908F907F906F905F904F9018
:1070C0003F902F90089580913D06882371F0109293
:1070D0003D0682E20E94901681E00E94E81D80E059
:1070E0000E94E81D80E00E94430290917804809104
:1070F000B6059817C9F0909078048091B6058093F2
:10710000780480917A04833009F4CEC580917A04A2
:10711000823050F08091B005882331F4E0917804FA
:10712000F0E0E854FA4F708286E10E94F71388235A
:1071300029F08091B005882309F474C580917A0400
:10714000833009F4C2C386E10E940D14882309F438
:10715000EFCC80917A04823009F0EACC70927A0404
:1071600080E00E94E81D82E00E949016E1CC8091B0
:107170003D06882361F010923D0682E20E9490163F
:107180008FE00E9458160E94671810927A0480912E
:10719000B5050E940D14882309F442C08091F805BA
:1071A0008093C40670923D0680917A04882391F5FD
:1071B0008091DD0630911E0720913A0690E0880FFD
:1071C000991F830F911D880F991F880F991F880F92
:1071D000991F280F209376048091400680937504B0
:1071E0008823C1F090E0A0E0B0E0282F30E02295A5
:1071F0003295307F3227207F3227FD01EC57F94F3F
:107200008081A650BA4F8C939F5FA92FB0E0A21740
:10721000B3079CF38FE00E9490168DE00E949016B9
:107220008DE00E94F713882309F482CC80917A04C0
:10723000882309F07DCC80917504882309F478CCEB
:1072400070927A048091DD0620911E0710913A0613
:1072500090E0880F991F820F911D880F991F880F4A
:10726000991F880F991F180F80917604181709F439
:107270005FCC8DE00E94581682E00E9458160E9452
:1072800067189091760480914006882309F442C0E3
:10729000A92EBB24A294B294B0EFBB22BA24AB2295
:1072A000BA247501C12EDD24C294D294A0EFDA2253
:1072B000DC24CA22DC2400E010E0C7010E94F71E93
:1072C000882E0C57194FF8018083C6010E94F71EC3
:1072D000B7010E94B31E882DB6010E94B31E82E042
:1072E0000E943C0F0E947C0C0894E11CF11C089445
:1072F000C11CD11C8E2D8A19082F10E080914006E8
:1073000090E082959295907F9827807F9827081724
:1073100019079CF210913A0684E896E00E94202A10
:10732000898389818F708F5F8093F7031093B705EE
:10733000898184FD73C58CE08093F50382E00E940F
:1073400090160E946718F4CB80913D068823E9F0DF
:1073500010923D060E94071782E20E945816709212
:10736000850481E20E94581680913A066091400699
:107370004091B3052091410600913A06E090B10595
:107380000E94561981E00E94430283E00E94361455
:10739000882309F445C080914106882309F02FC451
:1073A00090911E078091B105981781F08091B105E9
:1073B00080931E078091DD0660911E0740913A067A
:1073C0002091400604E816E00E94072D60914006D7
:1073D00084E896E04EED56E028EB35E00E948E2AD8
:1073E00080E090E0FC01E854FA4F1082019680346E
:1073F0009105C1F782E080937704109221071092E3
:1074000079041092780410927A041092B005709268
:107410007C0489E08093C40670923D0699249A9476
:107420008091C406843011F01092850480912B075E
:10743000882321F47092C40670923D0680918404E2
:10744000813009F075CB109284049091E80480910A
:10745000EE04891709F01FCE6BCB80913D0688237F
:10746000C9F010923D060E94071770927A0484E8D2
:1074700096E00E94202A282F2F702F5F20937804F7
:1074800090E0929582958F7089279F7089278170EF
:10749000809379048EE00E947515823009F4D4C07F
:1074A0008AE00E947515823009F4C5C089E00E9407
:1074B0007515823009F4B3C08FE00E94F71388235A
:1074C00091F030927A0480917904882311F44092EB
:1074D0007804809179048F5F809379048091790496
:1074E00081708093790480917A0480FF21C080911B
:1074F0007A04815080937A0480917904882309F476
:10750000ACC180917804803108F4CBC381E08093D2
:10751000780483E00E94581680917804882309F04B
:1075200099C181E080937804809178040E9440178B
:1075300080E00E940D14882309F4FACA80917A042D
:107540008230B8F182E08093770484E896E061E0CD
:107550004EED56E028EB35E00E948E2A909178049B
:1075600080917904811180E191509F70892B8093E3
:10757000C80684E896E061E04EED56E028EB35E081
:107580000E946F2B8091DD0660911E0740913A06A4
:1075900021E004E816E00E947C2D8091DD066091D8
:1075A0001E0740913A06209140060E94072D109236
:1075B00077047092C40670923D06BACA182F115013
:1075C000812F0E9446198091DD0690911E07E82EBA
:1075D000FF24EE0CFF1CE90EF11CEE0CFF1CEE0C60
:1075E000FF1CEE0CFF1CE10EF11CE294F29470EF14
:1075F000F722FE24E722FE248701005F1F4F8FE061
:10760000B7010E94B31E82E00E943C0F0E947C0CD6
:107610000894E11CF11CE016F10689F7C3CA8091B9
:10762000780490E00E968F7090708F5F809378044E
:1076300030927A0441CF809178048F708F5F80936D
:10764000780430927A0432CF80917A04823008F440
:10765000A3C3809178048F5F8093780430927A047A
:107660001FCFE92DF0E0E854FA4F508293948091B7
:107670007904981610F06624639470927A0410923C
:10768000780480917A0490E083709070892B09F4DB
:10769000B0CB0E941C17809140068823B1F090E087
:1076A00080E001C08E2FE92FF0E0E853F94FE08130
:1076B000EF70EF5FE80F981618F09E1608F4FDC201
:1076C0009F5F80914006981768F384E00E949016AF
:1076D00083E00E94901688E00E94901680917A04C0
:1076E00080FD13C0E2E05E1609F49AC3F1E05F1674
:1076F00009F49AC3552031F084E00E94581683E0C3
:107700000E94581688E00E9458160E94671810922E
:107710007A046FCB0E941C17E92DF0E0EE5BF94F65
:1077200080818F3FD1F0108112951F7000810F7002
:10773000010F0F5F101738F010C0812F0E945E17E5
:107740001F5F101750F480917A0480FDF6CF812FCF
:107750000E942A171F5F1017B0F380917A0480FFF0
:10776000DEC1882D60E00E94B11910927A040E9457
:107770006718B3CB86E10E94F713882309F0D9C2BA
:107780000E948C14882309F0A2C287E10E940D1484
:10779000882329F0FFE39F0E9F2270927A048EE0E7
:1077A0000E94F713882321F080E1882A70927A04DE
:1077B0008FE00E94F713882321F090E2892A7092CB
:1077C0007A0484E10E94F713882321F0E0E88E2AEE
:1077D00070927A0485E10E94F713882321F0F0E487
:1077E0008F2A70927A048EE00E940D14882321F073
:1077F0008FEE882270927A048FE00E940D14882305
:1078000021F09FED892270927A0484E10E940D1488
:10781000882321F0EFE78E2270927A0485E10E949E
:107820000D14882309F451CBFFEB8F2270927A0458
:107830004CCB86E10E943614882309F468CAE92DEE
:10784000F0E0E854FA4F50807092780482E0809320
:107850007A045DCA8091780465CE80917804813184
:1078600008F41CC281E08093780483E00E949016A3
:1078700053CE112309F009C280917804882309F4BA
:1078800004C2662029F4E92DF0E0E854FA4F508252
:1078900082E080937A0480917A04843009F09CCA53
:1078A000112359F080917804882339F493948091BE
:1078B0007904981610F06624639470927A048CCA46
:1078C0006092C40660923D0633C90E942415882345
:1078D00009F439CC82E080937A0486E10E94E113B6
:1078E000882309F030CC70927A040E94E81D2BCCDA
:1078F00088E00E940D14882309F4D8CA10927804F5
:1079000070927A0480917804813009F0D4CA86E1BB
:107910000E940D14882309F044C28EE00E94F713E0
:10792000882349F0882D809580719FEE8922882ACE
:1079300082E080937A048FE00E94F713882349F055
:10794000882D80958072EFED8E22882A82E08093C8
:107950007A0484E10E94F713882349F0882D8095EA
:107960008078FFE78F22882A82E080937A0485E17D
:107970000E94F713882349F0882D809580749FEB2F
:107980008922882A82E080937A040E948C14182F1E
:10799000882309F490CA80E00E94E81D82E00E94DA
:1079A0003C0F11501F70E0EF8E22812AE82DF0E08D
:1079B000EF73F070E750FC4F482D4078808160E015
:1079C0000E94D11D82E080937A04809178048330F4
:1079D00009F076CA0E948C14182F0E94A6148823DE
:1079E00019F4112309F46CCAE92DF0E0E252F94FC1
:1079F000808280E00E94E81D82E00E943C0F939408
:107A0000FFE3F91518F410927904992470927A041E
:107A1000109278048FE088228EE00E94E113882380
:107A200011F090E1892A8FE00E94E113882311F080
:107A3000E0E28E2A84E10E94E113882311F0F0E84D
:107A40008F2A85E10E94E113882311F080E4882ABF
:107A5000112309F435CA812E8A949FE089228EE091
:107A60000E94E113882311F0E0E18E2A8FE00E944A
:107A7000E113882311F0F0E28F2A84E10E94E113E0
:107A8000882311F080E8882A85E10E94E113882389
:107A900011F090E4892AE82DF0E0EF73F070E750E0
:107AA000FC4F482D4078808160E00E94D11D82E02B
:107AB00080937A043092780403CA86E10E940D1400
:107AC000882319F088E0809378048EE00E94F713F1
:107AD000882329F082E080937A0412E0512E8FE00F
:107AE0000E94F713882329F082E080937A045524BA
:107AF000539484E10E94F713882309F403C982E0B8
:107B000080937A045524FEC887E10E940D148823CF
:107B100009F4F3C81092780470927A04EEC8882DA4
:107B200061E00E94B11921CE82E00E9458160E94A5
:107B300067189091DD0620911E0730913A068091DA
:107B400075048823C9F1E92EFF24EE0CFF1CE20E18
:107B5000F11CEE0CFF1CEE0CFF1CEE0CFF1CE30EE8
:107B6000F11CE294F29460EFF622FE24E622FE2459
:107B70008701A0E0B0E0FD01E650FA4F8081AC57EC
:107B8000B94F8C93B8010E94B31E82E00E943C0F53
:107B90000E947C0C0F5F1F4F802F8E19A82FB0E022
:107BA0008091750490E082959295907F9827807FD0
:107BB0009827A817B907FCF210913A0684E896E0D6
:107BC0000E94202A898389818F708F5F8093F703B9
:107BD0001093B705898184FDE2C08CE08093F503A2
:107BE000CAC9992309F4ADC982E20E9490168DE0BA
:107BF0000E9458160E94671810927A04AAC98091B0
:107C0000F9058093DD068091B10580931E07809170
:107C1000B30580933A068091410680934006109206
:107C20004106C8CB82E080937A040E940E15882317
:107C300011F030927A04E0917804F0E0E854FA4FC1
:107C400082E08083E0917904F0E0E252F94F808095
:107C500080923E06E82DF0E0EF73F070E750FC4FA5
:107C6000482D4078808160E00E94D11D8091780489
:107C7000981639F090907804809179048F5F809302
:107C8000790482E00E94581659CA9394809179042D
:107C9000981608F4F6CD66246394FACD80917804A2
:107CA000E2CD8091780433CC0E940E15882309F030
:107CB0002DCA82E080937A0429CA992D981B80915D
:107CC0007A0480FF9DC0892F0E945E17FECC882E0B
:107CD0008A94EFE08E228EE00E94E113882311F057
:107CE000F0E18F2A8FE00E94E113882311F080E2F7
:107CF000882A84E10E94E113882311F090E8892A00
:107D000085E10E94E113882311F0E0E48E2AE82D3A
:107D1000F0E0EF73F070E750FC4F482D4078808121
:107D200060E00E94D11D82E080937A043092780452
:107D30002CCDE92DF0E0E252F94F80808EE00E94D8
:107D4000E113882311F0E0E18E2A8FE00E94E11315
:107D5000882311F0F0E28F2A84E10E94E113882346
:107D600011F080E8882A85E10E94E113882311F050
:107D700090E4892AE82DF0E0EF73F070E750FC4FB3
:107D8000482D4078808160E00E94D11D82E0809380
:107D90007A0470927804F4CC109278045ACC80E182
:107DA0001DCFE92DF0E0E252F94F80828EE00E9473
:107DB000E113882381F588248FE00E94E113882352
:107DC00011F080E2882A84E10E94E113882311F0F7
:107DD00090E8892A85E10E94E113882311F0E0E40C
:107DE0008E2A80E00E94E81D9394FFE3F91518F4B1
:107DF00010927904992470927A04109278048DCDAF
:107E0000892F0E942A1761CC81E08093C406809359
:107E10003D060C94753590E1892ECECF80E18CCA59
:107E200084E00E94581671CC83E00E9458166DCCF5
:107E30000F931F93CF93DF93EC01442319F18B0130
:107E400050E070E020E030E0F901E853F94F608144
:107E50006F706F5FD80190E0FE01E50FF11D80812A
:107E60008D939F5F5F5F9617B8F3760F2F5F3F4F3D
:107E7000005F1F4F241740F3872FDF91CF911F9191
:107E80000F91089570E0872FDF91CF911F910F918F
:107E90000895BF92CF92DF92EF92FF920F931F93BC
:107EA000CF93DF936B01B42E442369F17C0110E082
:107EB00000E0C0E0D0E0C7010E94202AFE01E853A4
:107EC000F94F808320812F702F5FD70190E08D9133
:107ED000F601E10FF11D80839F5F1F5F9217B8F3DA
:107EE000020F219680E190E0E80EF91ECB1518F301
:107EF000802FDF91CF911F910F91FF90EF90DF9036
:107F0000CF90BF90089500E0F3CFCF92DF92EF9231
:107F1000FF920F931F93DF93CF93CDB7DEB7C0547B
:107F2000D0400FB6F894DEBF0FBECDBF10927A04DA
:107F30001092780482E0809377044091400684E8B0
:107F400096E06E010894C11CD11CB6010E94493F05
:107F5000E82E809179048E1510F0109279048091AA
:107F600040068823C1F090E030E0E32FF0E0E853D2
:107F7000F94F20812F702F5F80E0E92FF0E0EE5B5A
:107F8000F94F80838F5F9F5F8217B8F33F5F8091C7
:107F90004006381750F30E94A61580912B078823BE
:107FA00009F4C9C184E00E94802AFF240E94A6151A
:107FB0000E947C0C1091C406113081F01430F1F154
:107FC0000E949E2C882391F70E946D2C0E94A6157A
:107FD0000E947C0C1091C406113081F70E94862A01
:107FE000882309F0F4C086E10E943614882329F022
:107FF00080917B04882309F088C18091C406813078
:1080000011F01092850480912B07882309F070C12C
:108010000E94CB298823A1F210927704C05CDF4F25
:108020000FB6F894DEBF0FBECDBFCF91DF911F9189
:108030000F91FF90EF90DF90CF9008950E94862AD5
:10804000882309F037C110E086E10E9436148823A6
:1080500009F0D0C087E10E943614882309F0E6C0F9
:1080600086E10E940D14882309F0FCC087E10E947C
:108070000D14882309F001C186E10E94F7138823BB
:1080800009F006C18EE00E94F713882339F08F2D86
:10809000809580719FEEF922F82A12E08FE00E940D
:1080A000F713882339F08F2D809580729FEDF92288
:1080B000F82A12E084E10E94F713882339F08F2D0B
:1080C000809580789FE7F922F82A12E085E10E94E6
:1080D000F713882339F08F2D809580749FEBF92258
:1080E000F82A12E00E948C14282F882361F08F2D2B
:1080F00090E08F7090700D9734F421502F7080EFC6
:10810000F822F22A12E088E00E94F713882309F48B
:108110004AC08F2D90E08F7090700D970CF4ECC0DA
:1081200090EFF92200E010E080917904F601E80F69
:10813000F11DF08240914006C60164E876E00E949D
:10814000183FE82E81E080937B040D301105BCF5CB
:108150008F2D61E00E94B11984E20E9458160E949E
:108160001C17E0917904F0E0EE5BF94F80810E94EA
:108170002A170E9467188091C406843011F010926B
:10818000850480912B07882309F4AEC08091840474
:10819000813009F015CF109284040E94CB298823E6
:1081A00009F40ECF39CF123009F4C9C0113019F7D4
:1081B0000F2D10E00F7010700D3011054CF28F2D47
:1081C00060E00E94B11984E20E949016C8CF0E941C
:1081D000071782E20E9458161093850481E20E94DC
:1081E000901680917B04882309F4A1C082E00E944C
:1081F0007416F9CE809179048F5F80937904809111
:1082000079046E2D0E9489499093790480917904B4
:10821000F601E80FF11DF08082E00E94581611E08F
:1082200087E10E943614882309F41ACF80917904DB
:108230006E2D70E090E00197860F971F0E94A9496C
:108240008093790480917904F601E80FF11DF080A4
:1082500080E00E94581611E086E10E940D148823E8
:1082600009F404CF82E00E9490160E94671887E10B
:108270000E940D14882309F4FFCE80E00E9490161E
:108280000E94671886E10E94F713882309F4FACE4A
:1082900080E00E94E113882309F4F4CE8091B605B2
:1082A0008093790480917904F601E80FF11DF08044
:1082B00011E0E8CE0E94071782E20E94581681E082
:1082C0008093850481E20E94581680917B04882364
:1082D000C1F082E00E94741680917904F601E80FE3
:1082E000F11DF08011E0B0CE81E00E94802A4ECFD7
:1082F00084E00E94802A8CCE8FE0F82E0FE010E000
:1083000013CF82E00E949016E7CF82E00E94901681
:108310008091DD0660911E0740913A06209140064B
:1083200004E816E00E947C2D10927B0466CE82E069
:108330000E94901658CE81E00E94802A36CE0F2DE2
:1083400010E00F701070F0CE3F924F925F926F92DC
:108350007F928F929F92AF92BF92CF92DF92EF92D5
:10836000FF920F931F93DF93CF93CDB7DEB7C05823
:10837000D0400FB6F894DEBF0FBECDBF10927A0486
:108380001092780482E08093770440914006B1E433
:10839000CB2ED12CCC0EDD1E84E896E0B6010E94D7
:1083A000493FF82E0E94A61580912B07882309F4D7
:1083B00059C684E00E94802A7724442466245524E8
:1083C00088248A949924332433945E010894A11C50
:1083D000B11C0E94A6150E947C0C1091C4061F308F
:1083E000B9F0103108F08AC0113009F4BAC2143063
:1083F00009F44EC20E949E2C882359F70E946D2CCE
:108400000E94A6150E947C0C1091C4061F3049F7EB
:108410000E94862A882309F09BC40E94F82B86E1DB
:108420000E94F713882309F08AC489E00E94F71399
:10843000882309F0D5C28AE00E94F713882309F047
:10844000C7C286E10E940D14882309F0BDC289E0ED
:108450000E940D14882309F0B3C28AE00E940D1413
:10846000882309F0A9C28DE00E94F713882329F020
:1084700080917504882309F05AC591E0791609F4B2
:10848000DBC3A2E07A1609F4D3C3B3E07B1609F08C
:10849000B1CF30927B04662D70E0842D992787FD43
:1084A0009095860F971F850D911D0E94A949582E02
:1084B000FF2099F020E030E0F601E20FF31F852D58
:1084C000820F662D0E948949D501A90FB11D8C919B
:1084D00080832F5F3F4F2F1578F340914006C601F0
:1084E00064E876E00E94183F4091400684E896E0F8
:1084F000B6010E94493FF82E77247CCF113109F450
:108500001BC1113108F480C0123109F073CF0E94F1
:10851000862A882309F056C40E94F82B8CE00E941A
:10852000F713882309F077C38CE00E940D14882389
:1085300009F06DC38EE00E94F713882309F05DC334
:108540008FE00E94F713882309F04DC384E10E9455
:10855000F713882309F03DC385E10E94F7138823B0
:1085600009F02DC388E00E94F713882309F01DC38A
:108570008EE00E940D14882309F0EFC28FE00E9464
:108580000D14882309F0F2C284E10E940D1488239F
:1085900009F0F5C285E10E940D14882309F0F8C2A4
:1085A00088E00E940D14882309F0FBC2772009F4AB
:1085B00021CF30927B04FF2009F48FCF860110C0B9
:1085C0000E97F9F08E2D8821D8019C919921892B45
:1085D000F80181938F018E2F8C198F1508F07DCFB4
:1085E0000E94FC00E82E90E08F7090708D30910515
:1085F00039F7E7EFEE228E2D90E08F7090700E9796
:1086000009F7F7EFEF22DECF0E94862A882309F0D0
:108610009EC20E94F82B8CE00E94F713882309F079
:10862000E7C187E10E94F713882309F0ECC180E0DD
:108630000E94F713882309F0F1C18CE00E940D1409
:10864000882309F0F6C187E10E940D14882309F000
:10865000F9C180E00E940D14882309F0FCC18EE06E
:108660000E94F713882309F0FFC18FE00E94F713DF
:10867000882309F008C284E10E94F713882309F0D7
:1086800011C285E10E94F713882309F01AC288E01D
:108690000E94F713882309F023C28EE00E940D1474
:1086A000882309F02CC28FE00E940D14882309F062
:1086B0002FC284E10E940D14882309F032C285E1A3
:1086C0000E940D14882309F035C288E00E940D1421
:1086D000882309F038C2772009F48CCE30927B04CD
:1086E000E2E07E1609F4D0C3F4E07F1609F46FC40B
:1086F000B1E07B1609F02CC4FF2009F4EECE860110
:1087000007C00F5F1F4F802F8C198F1508F0E5CE23
:108710000E94FC00E82EEFE1E81798F30E94FC00AD
:10872000D8012C916F2D0E948949F601E90FF11DA6
:1087300080818C932083E5CF0E94862A882309F0CC
:10874000F9C20E94F82B8CE00E94F713882309F0ED
:10875000E8C28CE00E940D14882309F0DEC28EE08E
:108760000E94F713882309F0CEC28FE00E94F7130E
:10877000882309F0BEC284E10E94F713882309F020
:10878000AEC285E10E94F713882309F09EC288E0FB
:108790000E94F713882309F08EC28EE00E940D1408
:1087A000882309F084C28FE00E940D14882309F009
:1087B0005FC284E10E940D14882309F062C285E142
:1087C0000E940D14882309F065C288E00E940D14F0
:1087D000882309F068C28DE00E94F713882329F0EE
:1087E00080917504882309F043C0172D10FF02CE35
:1087F00030927B0411FDEFC2FF2041F1860106C0DB
:108800000F5F1F4F802F8C198F1500F50E94FC0001
:10881000E82EBFE3B817A0F30E94FC00E82E90E01A
:108820008F7090708D30910509F404C30E9709F490
:10883000FEC29E2D9821D8018C918921982B9C9362
:108840000F5F1F4F802F8C198F1500F3BEEF7B2217
:1088500040914006C60164E876E00E94183F4091CE
:10886000400684E896E0B6010E94493FF82EC2CD4A
:10887000872D80958270B1E07B22782A8DE00E945E
:108880009016172D71FCCBC366240E946718AECFDB
:108890000E94862A882309F07FC284E00E94361451
:1088A000882309F072C285E00E943614882309F0FB
:1088B00065C282E10E943614882309F058C281E122
:1088C0000E943614882309F04BC286E10E943614B8
:1088D000882329F080917B04882309F016C387E15F
:1088E0000E943614882329F080917B04882309F0A4
:1088F000B2C28091C406843041F01092850482E0B7
:108900000E94901682E20E94901680912B07882385
:1089100009F48AC180918404813009F06BCD1092F2
:1089200084040E94CB29882309F464CD1092770433
:10893000C058DF4F0FB6F894DEBF0FBECDBFCF914A
:10894000DF911F910F91FF90EF90DF90CF90BF903C
:10895000AF909F908F907F906F905F904F903F90DF
:1089600008950E94862A882389F48091C406813064
:1089700011F01092850480912B07882309F027C2FB
:108980000E94CB29882309F435CDD0CF0E94071748
:1089900082E20E9458161093850481E20E9490168C
:1089A00080917B04882309F4CFC282E00E94741670
:1089B00081E00E944302D9CF8CE10E94901653CDF2
:1089C0008BE10E94901649CD82E00E9490163FCD27
:1089D0008CE10E9458167E2C73944424439431CD2C
:1089E0008BE10E9458167E2C739444244A9423CD24
:1089F0008EE00E9458167724739487E10E94F71343
:108A0000882309F414CE80E00E945816F2E07F2EED
:108A100080E00E94F713882309F40FCE82E20E94BF
:108A20005816E3E07E2E8CE00E940D14882309F492
:108A30000ACE8EE00E94901687E10E940D148823D2
:108A400009F407CE80E00E94901680E00E940D1489
:108A5000882309F404CE82E20E9490168EE00E94E0
:108A6000F713882309F401CE84E00E94581674E0BD
:108A7000772E60E1862E5FEE952E8FE00E94F71331
:108A8000882309F4F8CD83E00E94581644E0742E40
:108A900030E2832E2FED922E84E10E94F71388237B
:108AA00009F4EFCD88E00E94581694E0792E80E812
:108AB000882E0FE7902E85E10E94F713882309F492
:108AC000E6CD81E00E94581614E0712EB0E48B2EA2
:108AD000AFEB9A2E88E00E94F713882309F4DDCDCE
:108AE00084E20E945816F4E07F2EEFE08E2E70EFA5
:108AF000972E8EE00E940D14882309F4D4CD84E0D3
:108B00000E9490168FE00E940D14882309F4D1CDA5
:108B100083E00E94901684E10E940D14882309F4DA
:108B2000CECD88E00E94901685E10E940D14882326
:108B300009F4CBCD81E00E94901688E00E940D14CC
:108B4000882309F4C8CD84E20E949016C4CD89E13F
:108B50000E945816772444245CCD84E00E9490162D
:108B60008FE00E940D14882309F40ECD83E00E944B
:108B7000901684E10E940D14882309F40BCD88E03F
:108B80000E94901685E10E940D14882309F408CDF7
:108B900081E00E94901688E00E940D14882309F459
:108BA00005CD84E20E94901601CD84E20E94581601
:108BB000772473942FE0822E90EF992ED9CC81E008
:108BC0000E9458167724739440E4842E3FEB932E32
:108BD000C9CC88E00E9458167724739460E8862EEA
:108BE0005FE7952EB9CC83E00E94581677247394E2
:108BF000E0E28E2E7FED972EA9CC84E00E945816DD
:108C000077247394A0E18A2EFFEE9F2E99CC8EE0FC
:108C10000E9490168FCC8EE00E9458167724739491
:108C200088248A94992480CC81E00E94802A72CE84
:108C3000442009F02ECCDECB442009F4DBCB70922B
:108C40007B04FF2089F0342D3F0DD60120E0822FD8
:108C5000830F6F2D0E948949F501E90FF11D8D9158
:108C600080832F5F2F1598F340914006C50138CCC3
:108C700083E00E94901684E10E940D14882309F479
:108C80009ECD88E00E94901685E10E940D148823F5
:108C900009F49BCD81E00E94901688E00E940D149B
:108CA000882309F498CD84E20E94901694CD84E044
:108CB0000E94901678CD84E20E945816A1E07A2A8C
:108CC0001FE0812EB0EF9B2E68CD81E00E945816E8
:108CD00091E0792A80E4882E0FEB902E58CD88E021
:108CE0000E94581681E0782A20E8822E9FE7992E6C
:108CF00048CD83E00E945816F1E07F2A40E2842E9E
:108D00003FED932E38CD84E00E945816E1E07E2A94
:108D100060E1862E5FEE952E28CD8EE00E949016A3
:108D20001ECD8EE00E945816B1E07B2A88248A94DA
:108D300099240FCD8CE00E945816772402CD82E052
:108D40000E9458164090B6054194772473946DCBD9
:108D500080E20E94581677244424EE2455245DCBEB
:108D60006091C40681E141E10E946C2AAECD609120
:108D7000C40682E142E10E946C2AA1CD6091C40642
:108D800080E145E00E946C2A94CD6091C4068FE09A
:108D900044E00E946C2A87CD0E94071782E20E945D
:108DA00058163092850481E20E94581680917B0407
:108DB000882309F4A6C082E00E94741681E00E9414
:108DC00043026BCD8BE00E9458167724A5CB84E03C
:108DD0000E94802AD5CDFF2009F438CD860107C036
:108DE0000F5F1F4F802F8C198F1508F02FCD0E9419
:108DF000FC00E82EEFE3E81798F30E94FC00662DD4
:108E00000E948949F501E90FF11DE0808E2D90E067
:108E10008F7090708D309105B9F00E9791F09E2D66
:108E20009821D8018C918921982B9C93D9CFF7EF69
:108E3000EF22FFCCE7EFEE228E2D90E08F70907046
:108E4000F5CC87EFE822EBCFF7EFEF228E2D90E005
:108E50008F709070E2CF82E00E9490168091DD06C4
:108E600060911E0740913A062091400604E816E002
:108E70000E94072D40914006C801B6010E94493F5B
:108E8000F82E10927B0435CD6F2D6695D9F09F2D6D
:108E9000915040E050E0A92FB0E09501240F351F1C
:108EA000F601EA0FFB1F8081F9018083AA0DBB1D2B
:108EB000F601E40FF51F80818C9391504F5F5F4F57
:108EC000461748F3FF2009F408CB81E040E050E06A
:108ED0006F2D0E948949D601A40FB51FF501E90F36
:108EE000F11D20812074F501E40FF51F80818F7B37
:108EF000282B2C93892F8F5F4F5F5F4F4F1540F3C7
:108F0000ECCA82E00E94901659CF82E00E9490162F
:108F10008091DD0660911E0740913A06209140063F
:108F200004E816E00E947C2D10927B04D8CCE394D8
:108F300081E0E8228DE00E949016EE2009F07BC0CF
:108F400066240E94671899CA82E00E94901630CD6C
:108F50006091400684E896E0A60128EB35E00E9487
:108F60008E2AF82E882311F1860106C00F5F1F4F4D
:108F7000802F8C198F15D0F40E94FC00E82EBFE3DF
:108F8000B817A0F30E94FC00F80120816F2D0E9409
:108F90008949F601E90FF11D8081D8018C93208366
:108FA0000F5F1F4F802F8C198F1530F36091400693
:108FB00084E896E0A60128EB35E00E946F2B4091F3
:108FC000400684E896E0B6010E94493F86CAFF2029
:108FD00009F483CA860107C00F5F1F4F802F8C19C9
:108FE0008F1508F07ACA0E94FC00E82E8FE38E15D8
:108FF00098F30E94FC00D8012C916F2D0E948949A2
:10900000F601E90FF11D80818821992D9223892B8A
:109010008C93808189212821822B8083DDCF8DE074
:109020000E9458168AEF95E0B501409175040E94A0
:10903000493F682E2ACC8DE00E9458168AEF95E0B1
:10904000B501409175040E94493F682E4091400649
:1090500084E896E0B6010E94493FF82EA3E07A2EFC
:1090600044246FCF81E00E94802AA6C9EF920F931B
:109070001F930E94A61580912B07882309F426C10F
:1090800084E00E94802A07C0113009F47EC00E944B
:109090009E2C8823E1F00E94A6150E947C0C109162
:1090A000C4061330F1F0143078F3143009F447C0DB
:1090B0001D3069F781E00E94B0338091C4068D3085
:1090C00031F3109285040E949E2C882321F70E9480
:1090D0006D2C0E94A6150E947C0C1091C4061330C2
:1090E00011F70E94862A882309F09AC00E94F82B63
:1090F000882321F010927704109285040E948C142A
:10910000882309F07AC080912B07882309F0BFCF0C
:1091100086E10E94F713882309F4B9CF80E00E940A
:10912000E81D81E00E943C0F80E00E94642A90913B
:10913000CC06890F60E040E00E94D11DA8CF0E94BC
:10914000862A882309F081C080E00E94B0338823FA
:1091500009F478C08091C406843011F0109285041F
:1091600080912B07882309F48DC08091840481307D
:1091700009F08DCF109284040E94CB29882309F432
:1091800086CF1F910F91EF9008950E94862A882321
:1091900009F07CC080E00E94B033182F86E10E9465
:1091A000F7138823C9F41123A1F08091C4068130FC
:1091B00011F01092850480912B07882309F082C05A
:1091C0000E94CB29882309F462CF1F910F91EF9061
:1091D00008950E948B2CE9CF80E00E94E81D81E079
:1091E0000E943C0F80E00E94642A9091CC06890F77
:1091F00060E040E00E94D11DD6CF182F11500E9490
:109200004718812F0E941E181093C50680912B07C6
:10921000882309F078CF8091C5068093CC0673CF60
:109220000E94071711E01093770481E00E94430227
:1092300084E20E9458168091C5060E941E18109361
:10924000850454CF0E948B2C85CF0E94071782E2A1
:109250000E94581681E08093850481E20E9458168E
:1092600080913A06609140064091B30520914106F5
:1092700000913A06E090B1050E94561981E00E94E3
:10928000430262CF81E00E94802A6FCF0E940717BD
:1092900082E20E9458161093850481E20E94901683
:1092A00080913A06609140064091B30520914106B5
:1092B00000913A06E090B1050E94561981E00E94A3
:1092C000430268CF84E00E94802A7ACF81E00E9426
:1092D000802AE1CE629FD001739FF001829FE00D52
:1092E000F11D649FE00DF11D929FF00D839FF00D25
:1092F000749FF00D659FF00D9927729FB00DE11DD1
:10930000F91F639FB00DE11DF91FBD01CF011124AD
:109310000895991B79E004C0991F961708F0961BD1
:10932000881F7A95C9F780950895AA1BBB1B51E148
:1093300007C0AA1FBB1FA617B70710F0A61BB70BC5
:10934000881F991F5A95A9F780959095BC01CD016A
:10935000089597FB092E07260AD077FD04D0E5DF94
:1093600006D000201AF4709561957F4F0895F6F7A6
:10937000909581959F4F0895A1E21A2EAA1BBB1BC1
:10938000FD010DC0AA1FBB1FEE1FFF1FA217B307D1
:10939000E407F50720F0A21BB30BE40BF50B661FE7
:1093A000771F881F991F1A9469F7609570958095AB
:1093B00090959B01AC01BD01CF010895F894FFCFBA
:1093C00001FFFFFFFFFFFFFFFFD0121300000100AE
:1093D0000100010001000100010001000100010085
:1093E00001000100010001C000800040007F2064F6
:1093F00030480F04050607111210130E0405060766
:10940000111210130409050A06070B110C120D1096
:109410001325212326272422201D1E1B191F1C1A59
:109420001012180F110C130E0B140D0A1516091734
:109430000405080306010700020320191A180C0B83
:109440000A090420191A180C0B0A092221252320C5
:10945000191A18241B1C0F0E0D04030A0C0B090803
:10946000010200201B191C1A180F0C0E0B0D0A0903
:1094700026271D1E1F101211131415161705060797
:109480006E306E783078000100070E091C1B121533
:10949000383F363124232A2D70777E796C6B6265D4
:1094A000484F464154535A5DE0E7EEE9FCFBF2F5C4
:1094B000D8DFD6D1C4C3CACD90979E998C8B8285B4
:1094C000A8AFA6A1B4B3BABDC7C0C9CEDBDCD5D2A4
:1094D000FFF8F1F6E3E4EDEAB7B0B9BEABACA5A294
:1094E0008F88818693949D9A2720292E3B3C353284
:1094F0001F18111603040D0A5750595E4B4C454274
:109500006F68616673747D7A898E878095929B9C63
:10951000B1B6BFB8ADAAA3A4F9FEF7F0E5E2EBEC53
:10952000C1C6CFC8DDDAD3D4696E676075727B7C43
:1095300051565F584D4A4344191E171005020B0C33
:1095400021262F283D3A33344E49404752555C5B23
:109550007671787F6A6D64633E39303722252C2B13
:109560000601080F1A1D1413AEA9A0A7B2B5BCBB03
:109570009691989F8A8D8483DED9D0D7C2C5CCCBF3
:10958000E6E1E8EFFAFDF4F30409050A06070B111A
:109590000C120D1013000100010001000100010078
:1095A000010001000100010001000100010001C0F3
:1095B0000080004000060601011718191A1B1C1D27
:1095C0001E1F202122233F3F3F0B0C0D0E0F1011B9
:1095D0001213141516173F3F3F2324252627282949
:1095E0002A2B2C2D2E2F3F3F3F1718191A1B1C1DFD
:0C95F0001E1F202122233F3F3F150000DA
:00000001FF
